:10000000A2C20000D1C20000CFC20000CDC20000D9
:10001000CBC20000C9C20000C7C20000C5C20000B8
:10002000C3C20000C1C20000BFC20000BDC20000C8
:10003000BBC20000B9C20000B7C20000B5C20000D8
:10004000B3C200000C94482FAFC20000ADC2000044
:100050000C948B31A9C20000A7C200000C946D2D36
:10006000A3C200000C94902B0C94672B9DC200003F
:100070009BC2000099C2000097C2000095C2000018
:100080000C941B2F91C200008FC200008DC2000093
:100090008BC2000089C2000087C2000085C2000038
:1000A00083C2000081C200000C94EE2E7DC20000CD
:1000B0007BC2000079C2000077C200000C94C12E00
:1000C00073C2000071C200006FC200006DC2000068
:1000D0006BC2000069C2000067C2000065C2000078
:1000E00063C20000E002ED02F602FF020C031503FA
:1000F000B106B106B106B106B10622032F033C03D7
:10010000B106490352035B03680371037A03830357
:100110008C039503B1069E03A703B003B106B10695
:10012000B106B903C203CB03B106B106D403E103A0
:10013000B106B106B106EE03FB030804B1061504CF
:100140001E042704B106B106B10630043904420486
:10015000B1064F045C046904B106B106B106760429
:1001600083049004B1069D04AA04B704B106B10645
:10017000B106C404D104DE04B106EB04F404FD04AA
:10018000B106B106B106B106B106B106B106B106B7
:10019000B106B106B106B106B106B106B106B106A7
:1001A000B106B106B106B106B106B106B106210528
:1001B0002A053305B1063C0545054E05B106B106D5
:1001C000B106570564057105B1067E058B059805D6
:1001D000B106B106B106A505B205BF05B106CC054D
:1001E000D505DE05B106B106B106E705F005F9054E
:1001F000B106B106B106B106B106B106B106B10647
:10020000B106B106B10606050F051805B106B1061F
:10021000B106B106B106B106B106B106B106B10626
:10022000B106B106B106B106B106B106B106B10616
:10023000B106B106B106B106B106B106B106B10606
:10024000B106B106B106B106B106B106B106B106F6
:10025000B106B106B106B106B106B106B106B106E6
:10026000B106B106B106B106B106B106B106B106D6
:10027000B106B106B10602060B061806B106250640
:100280002E063B06B106B106B106480651065E06CB
:10029000B1066B0674068106B106B106B1068E067C
:1002A0009706A406FF080409090913091D09960900
:1002B00027092F09370941094B09550964096E09B6
:1002C0009609780982098C095C295F294E295229EF
:1002D00058299629632967296D29712975297B2950
:1002E0007F298329962989298D2991294E414E49B3
:1002F0004E495459494E46CDCCCC3D0AD7233C17E4
:10030000B7D13877CC2B329595E6241FB14F0A0030
:100310000020410000C84200401C4620BCBE4CCA20
:100320001B0E5AAEC59D7400407A10F35A00A0729D
:100330004E18090010A5D4E80000E8764817000020
:10034000E40B54020000CA9A3B000000E1F50500EE
:100350000080969800000040420F000000A0860137
:10036000000000102700000000E803000000006407
:1003700000000000000A0000000000010000000072
:10038000002C76D888DC674F0823DFC1DFAE59E147
:10039000B1B796E5E3E453C63AE651997696E8E6B6
:1003A000C28426EB898C9B62ED407C6FFCEFBC9C89
:1003B0009F40F2BAA56FA5F490055A2AF75C936B9B
:1003C0006CF9676DC11BFCE0E40D47FEF520E6B556
:1003D00000D0ED902E0300943577050080841E0830
:1003E0000000204E0A000000C80C333333330F984E
:1003F0006E12831141EF8D2114893BE65516CFFE15
:10040000E6DB18D1844B381BF77C1D901DA4BBE4A0
:1004100024203284725E228100C9F124ECA1E53DE2
:100420002700002100240027002A002D003000337F
:100430000001010000040107010A0101021020204F
:100440000808102040102040800201020108040228
:10045000010102040810204080804020100804029E
:1004600001800402018040201008040201080402F7
:1004700001010204081020408001020408102040FD
:100480008005050505070508080808020202020A9A
:100490000A08080404040401010101010101010327
:1004A00003030303030303040707070C0C0C0C0CE2
:1004B0000C0C0C0202020206060606060606060BD5
:1004C0000B0B0B0B0B0B0B00000A0B02090C0D0E98
:1004D0000807030401000000000000000000000005
:1004E000000000000000000000000000000000000C
:1004F00000000012111000000000000000000000C9
:1005000000000000000000000000000000000022C9
:1005100000250028002B002E0031003400020100CD
:1005200000050108010B010000200023002600291E
:10053000002C002F00320000010000030106010919
:100540000100D548D14811241FBECFEFD1E2DEBF54
:10055000CDBF00E00CBF17E0A0E0B2E0ECEBF5EAA5
:1005600000E00BBF02C007900D92A434B107D9F789
:100570002CE0A4E4B7E001C01D92A53FB207E1F76B
:1005800012E0C2EAD2E000E006C021970109802F04
:10059000FE010E94C051C13AD10780E00807A9F7C7
:1005A0000E94203E0C94CD522BCD603E710508F088
:1005B000D8C3FB018827EE58FF4F8F4F0C94C051D2
:1005C00081E090E0A0E0B0E0809358079093590755
:1005D000A0935A07B0935B07089510925C0710929E
:1005E0005D0710925E0710925F07089510926007F2
:1005F000109261071092620710926307089581E0DC
:1006000090E0A0E0B0E08093640790936507A0932A
:100610006607B093670708951092680710926907FC
:1006200010926A0710926B07089583E090E0A0E0B3
:10063000B0E080936C0790936D07A0936E07B09322
:100640006F07089588E790E0A0E0B0E0809384070A
:1006500090938507A0938607B0938707089588E74E
:1006600090E0A0E0B0E08093880790938907A09382
:100670008A07B0938B07089588E790E0A0E0B0E088
:1006800080938C0790938D07A0938E07B0938F076C
:100690000895109294071092950710929607109261
:1006A00097070895109298071092990710929A0749
:1006B00010929B07089581E090E0A0E0B0E0809365
:1006C0009C0790939D07A0939E07B0939F07089562
:1006D0001092A0071092A1071092A2071092A307F0
:1006E00008951092A4071092A5071092A6071092E1
:1006F000A70708951092A8071092A9071092AA07B9
:100700001092AB0708951092AC071092AD071092AB
:10071000AE071092AF0708951092B0071092B1077C
:100720001092B2071092B30708951092B407109276
:10073000B5071092B6071092B70708951092BC073C
:100740001092BD071092BE071092BF070895109235
:10075000C0071092C1071092C2071092C3070895F4
:100760001092C4071092C5071092C6071092C707CF
:1007700008951092D4071092D5071092D6071092C0
:10078000D70708951092D8071092D9071092DA0768
:100790001092DB0708951092DC071092DD0710928B
:1007A000DE071092DF07089581E090E0A0E0B0E05E
:1007B0008093E8079093E907A093EA07B093EB07CB
:1007C000089581E090E0A0E0B0E08093EC07909382
:1007D000ED07A093EE07B093EF0708958CE291E048
:1007E000A0E0B0E08093FC079093FD07A093FE0784
:1007F000B093FF0708958CE291E0A0E0B0E0809311
:10080000000890930108A0930208B093030808958C
:100810008CE291E0A0E0B0E080930408909305089A
:10082000A0930608B0930708089510920C08109240
:100830000D0810920E0810920F08089510921008DB
:100840001092110810921208109213080895109235
:10085000140810921508109216081092170808959F
:10086000109224081092250810922608109227084A
:100870000895109228081092290810922A081092C0
:100880002B08089581E090E0A0E0B0E080932C0870
:1008900090932D08A0932E08B0932F08089585E01B
:1008A00090E0A0E0B0E08093340890933508A093E6
:1008B0003608B0933708089585E090E0A0E0B0E0F6
:1008C0008093380890933908A0933A08B0933B0876
:1008D000089589E190E0A0E0B0E080933C08909317
:1008E0003D08A0933E08B0933F08089582E390E04E
:1008F000A0E0B0E080934C0890934D08A0934E0880
:10090000B0934F08089582E390E0A0E0B0E08093B8
:10091000500890935108A0935208B093530808953B
:1009200082E390E0A0E0B0E08093540890935508F3
:10093000A0935608B0935708089582E390E0A0E092
:10094000B0E080935C0890935D08A0935E08B0933C
:100950005F08089582E390E0A0E0B0E08093600833
:1009600090936108A0936208B0936308089582E3AE
:1009700090E0A0E0B0E08093640890936508A093B5
:100980006608B0936708089580E991E0A0E0B0E0C0
:100990008093740890937508A0937608B0937708B5
:1009A000089580E991E0A0E0B0E08093780890930A
:1009B0007908A0937A08B0937B08089580E991E0C4
:1009C000A0E0B0E080937C0890937D08A0937E081F
:1009D000B0937F08089510928408109285081092B1
:1009E0008608109287080895109288081092890846
:1009F00010928A0810928B08089510928C08109219
:100A00008D0810928E0810928F08089510929C09FC
:100A100010929D0910929E0910929F0908951092BC
:100A2000A0091092A1091092A2091092A309089599
:100A30001092A4091092A5091092A6091092A70974
:100A400008951092EC081092ED081092EE081092A2
:100A5000EF0808951092F0081092F1081092F20831
:100A60001092F30808951092F4081092F50810926D
:100A7000F6081092F70808951092FC081092FD08ED
:100A80001092FE081092FF0808951092000910922B
:100A900001091092020910920309089510920409A5
:100AA000109205091092060910920709089585E031
:100AB00090E0A0E0B0E08093140990931509A09312
:100AC0001609B0931709089585E090E0A0E0B0E022
:100AD0008093180990931909A0931A09B0931B09E0
:100AE000089585E090E0A0E0B0E080931C09909329
:100AF0001D09A0931E09B0931F09089584EB95E189
:100B0000A0E0B0E08093240990932509A0932609E2
:100B1000B0932709089584EB95E1A0E0B0E08093BD
:100B2000280990932909A0932A09B0932B090895C5
:100B300084EB95E1A0E0B0E080932C0990932D091F
:100B4000A0932E09B0932F09089585E090E0A0E0CE
:100B5000B0E080933C0990933D09A0933E09B09387
:100B60003F09089585E090E0A0E0B0E0809340095F
:100B700090934109A0934209B0934309089585E0F9
:100B800090E0A0E0B0E08093440990934509A093E1
:100B90004609B0934709089510924C0910924D09E7
:100BA00010924E0910924F09089510925009109218
:100BB0005109109252091092530908951092540944
:100BC00010925509109256091092570908951092E3
:100BD00064091092650910926609109267090895D8
:100BE000109268091092690910926A0910926B09B3
:100BF000089510926C0910926D0910926E0910926E
:100C00006F09089510927C0A10927D0A10927E0A54
:100C100010927F0A08958CE390E0A0E0B0E080930A
:100C2000800A9093810AA093820AB093830A089560
:100C300081E090E0A0E0B0E08093840A9093850A80
:100C4000A093860AB093870A089510928C0A109296
:100C50008D0A10928E0A10928F0A08958CE390E00C
:100C6000A0E0B0E08093900A9093910AA093920A3A
:100C7000B093930A089581E090E0A0E0B0E0809303
:100C8000940A9093950AA093960AB093970A0895B0
:100C90001092A40A1092A50A1092A60A1092A70A0E
:100CA00008958CE390E0A0E0B0E08093A80A9093D0
:100CB000A90AA093AA0AB093AB0A089581E090E034
:100CC000A0E0B0E08093AC0A9093AD0AA093AE0A86
:100CD000B093AF0A08951092B40A1092B50A109218
:100CE000B60A1092B70A08958CE390E0A0E0B0E055
:100CF0008093B80A9093B90AA093BA0AB093BB0A3A
:100D0000089581E090E0A0E0B0E08093BC0A909369
:100D1000BD0AA093BE0AB093BF0A08951092CC0AF0
:100D20001092CD0A1092CE0A1092CF0A08958CE349
:100D300090E0A0E0B0E08093D00A9093D10AA09315
:100D4000D20AB093D30A089581E090E0A0E0B0E029
:100D50008093D40A9093D50AA093D60AB093D70A69
:100D60000895660F771F660F771FFB01E85AF84F4B
:100D7000108211821282138208950F931F93CF93D2
:100D8000DF938C01C0E0D0E0BE01C8010E940637AD
:100D9000882319F0BE01C80108DC2196C13ED105A7
:100DA00099F7DF91CF911F910F910895EF92FF92E4
:100DB0000F931F93CF93DF9300D01F92CDB7DEB771
:100DC0008B017B01EE0CFF1C622FC70129833A8344
:100DD0004B835C830E94345029813A814B815C8132
:100DE000992757FD9A95852F742F632FC701019678
:100DF0000E9434500D58110929813A814B815C8140
:100E000003301105A8F4BA01992777FD9095892F31
:100E1000C70144960E94345029813A814B815C81FC
:100E2000652F772788279927C70145960E94345058
:100E300080E090E00F900F900F900F90DF91CF9196
:100E40001F910F91FF90EF9008954F925F926F92D4
:100E50007F928F929F92AF92BF92CF92DF92EF924A
:100E6000FF92CF93DF935B01EB01CC0FDD1FCE012F
:100E70000E942C50482E512C612C712CCE010196D1
:100E80000E942C50C82ED12CE12CF12C8DE8A81AF0
:100E9000B10883E0A816B10488F5CE0144960E94FB
:100EA0002C50882E912CA12CB12CCE0145960E945D
:100EB0002C50482F50E060E070E08FEF88169104CE
:100EC000A104B104A9F44F3F51056105710581F4F6
:100ED0008FEF481651046104710481F48FEFC81636
:100EE000D104E104F10451F46FEF7FEFCB012BC08B
:100EF00040385105610571056CF0F6CF80E8C816E1
:100F0000D104E104F10484F740E050E0BA01812CFF
:100F1000912C5401FE2CED2CDC2CCC24C40CD51CC3
:100F2000E61CF71C540199248824C80CD91CEA1C1F
:100F3000FB1C742F662755274427CB01BA016C0D83
:100F40007D1D8E1D9F1DDF91CF91FF90EF90DF9053
:100F5000CF90BF90AF909F908F907F906F905F9059
:100F60004F9008950E94801BFC01148680E090E061
:100F700008958FE994E00E94C33C87E193E00E94CA
:100F8000C33C0E94801B0E948A1A80E090E0089572
:100F900080918D0B81113FC081E080938D0B0E9469
:100FA000FA19FC01E159FF4F2081222369F0709763
:100FB00040815181628173814F5F5F4F6F4F7F4FDF
:100FC0004083518362837383FC01E751FF4F20818B
:100FD000222369F0709740815181628173814F5F54
:100FE0005F4F6F4F7F4F4083518362837383FC0158
:100FF000ED59FE4F2081222361F07097808191810D
:10100000A281B3810196A11DB11D80839183A2832A
:10101000B38310928D0B08950C94FE490C94FE49F5
:101020000C94FE490C94FE490C94FE490C94FE4924
:101030000C94FE490C94FE490C94FE490C94FE4914
:101040000C94FE490C94FE490C94FE490C94FE4904
:10105000CF93DF93EB0120E030E040E85FE36A816B
:101060007B818C819D810E94104F811111C084EA87
:1010700094E00E94C33C0E94FA19FC01E25BFF4F1E
:10108000108211821282138282589E4F0E940A3E61
:1010900020E030E040E85FE36E817F8188859985BC
:1010A0000E94104F811111C084EB94E00E94C33C58
:1010B0000E94FA19FC01E853FF4F1082118212823C
:1010C000138284569E4F0E940A3E20E030E040E8A2
:1010D0005FE36A857B858C859D850E94104F811119
:1010E00011C084EC94E00E94C33C0E94FA19FC01F8
:1010F000EE5BFE4F108211821282138286549E4F45
:101100000E940A3E0E94801B0E948A1A80E090E0A2
:10111000DF91CF9108958F929F92AF92BF92CF921D
:10112000DF92EF92FF920F931F930E94FA1921E032
:101130002F931F921F921F921F92812C912CA12CF2
:10114000B12CC12CD12C760197018601B701A601E3
:101150008AD40F900F900F900F900F9080E090E046
:101160001F910F91FF90EF90DF90CF90BF90AF90C5
:101170009F908F9008950F931F93CF93DF938B01D0
:10118000EA01AB01415051094433510508F0D4C084
:101190002230310508F0D0C048E3429FF001439F60
:1011A000F00D1124E60FF71FE80FF91F81E080838F
:1011B000232B11F46C2F07C061E0802F0E94E22CDA
:1011C000209739F460E0802F0E94EE2B80E090E0C1
:1011D000B5C0CF3FD10509F4ADC0F801E953FB4FCD
:1011E000E4918E2F90E0FC013197E231F10508F097
:1011F0009DC08827EE5AFE4F8F4F0C94C05184B586
:10120000806884BDC7BDE2CF84B5806284BDC8BD9F
:10121000DDCF80918000806880938000D09389002A
:10122000C0938800D3CF809180008062809380003B
:10123000D0938B00C0938A00C9CF809180008860D2
:1012400080938000D0938D00C0938C00BFCF80919D
:10125000B00080688093B000C093B300B7CF809196
:10126000B00080628093B000C093B400AFCF809193
:101270009000806880939000D0939900C09398006C
:10128000A5CF80919000806280939000D0939B00C6
:10129000C0939A009BCF80919000886080939000CB
:1012A000D0939D00C0939C0091CF8091A000806856
:1012B0008093A0008091A0008F7B8093A000D093AA
:1012C000A900C093A80082CF8091A0008062809383
:1012D000A000D093AB00C093AA0078CF8091A0006B
:1012E00088608093A000D093AD00C093AC006ECF17
:1012F00080912001806880932001D0932901C093C0
:10130000280164CF80912001806280932001D093D6
:101310002B01C0932A015ACF8091200188608093CD
:101320002001D0932D01C0932C0150CFC038D1059E
:101330000CF448CF61E047CF81E090E0DF91CF919E
:101340001F910F9108958F929F92AF92BF92CF926B
:10135000DF92EF92FF920F931F930E94FA1960E0C1
:1013600070E00E949F37892BC9F40E94FA191F92DE
:101370001F9221E02F931F921F92812C912CA12C60
:10138000B12CC12CD12C760197018601B701A601A1
:101390006AD30F900F900F900F900F9080E090E025
:1013A0001F910F91FF90EF90DF90CF90BF90AF9083
:1013B0009F908F9008958F929F92AF92BF92CF92FD
:1013C000DF92EF92FF920F931F930E94FA1961E050
:1013D00070E00E949F37892BC9F40E94FA191F926E
:1013E00021E02F931F921F921F92812C912CA12CF0
:1013F000B12CC12CD12C760197018601B701A60131
:1014000032D30F900F900F900F900F9080E090E0EC
:101410001F910F91FF90EF90DF90CF90BF90AF9012
:101420009F908F900895CF92DF92EF92FF92CF938B
:10143000DF93EB010E940637882359F1FE01EE0F7E
:10144000FF1FEE0FFF1FE85AF84FC080D180E280E7
:10145000F38084ED94E00E94C33C82EA94E00E9411
:10146000C33C88ED94E00E94C33CCE010E94363D0F
:1014700082EA94E00E94C33C8AED94E00E94C33C5F
:10148000C701B6010E940F3D0E94801B0E948A1A6C
:1014900004C08CED94E00E94C33C80E090E0DF91BA
:1014A000CF91FF90EF90DF90CF900895EF92FF9251
:1014B0000F931F93CF93DF9380918E0B90918F0B9F
:1014C000892B09F066C084E090E00E946949EC0134
:1014D00060E070E0BADC16161706FCF0CE014DDCB9
:1014E00098E5E92E97E0F92E00E010E0B801CE0172
:1014F0000E940637882341F0F70120813181428123
:101500005381B801CE0152DC0F5F1F4FF4E0EF0EA4
:10151000F11C0639110551F738C063E070E0CE01C7
:1015200094DC613071058105910569F588E5E82E47
:1015300087E0F82E00E010E0B801CE010E940637E7
:101540008823C1F0B801CE0180DCF701608371838C
:10155000828393836F3F7F4F8F4F9F4F59F4B80122
:10156000CE0123D8F7012081318142815381B80116
:10157000CE011CDC0F5F1F4FF4E0EF0EF11C013EAB
:101580001105D1F602C0CE01F8DBD0938F0BC093CA
:101590008E0B80918E0B90918F0BDF91CF911F91CD
:1015A0000F91FF90EF900895EF92FF920F931F938A
:1015B000CF93DF9300D01F92CDB7DEB7FB0122A1FE
:1015C00033A144A155A1068D178D29833A834B83FE
:1015D0005C836CDF7C01FC018281938129813A81EB
:1015E0004B815C818F30F7E29F072CF40196F70165
:1015F0009383828303C0F70113821282B801C7016B
:1016000029833A834B835C830E94063729813A8180
:101610004B815C81882391F0F801EE0FFF1FEE0FE4
:10162000FF1FE85AF84F2083318342835383B80168
:10163000C701BCDBB801C701F6DE04C08CED94E045
:101640000E94C33C0E94421E0E940D1E80E090E05A
:101650000F900F900F900F90DF91CF911F910F91EE
:10166000FF90EF9008950F931F93CF93DF931EDFAA
:101670008C01C0E0D0E0BE01C8010E94063788237B
:1016800019F0BE01C801CFDE2196C13ED10599F700
:101690008EEF94E00E94C33C0E94801B0E948A1A35
:1016A00080E090E0DF91CF911F910F910895089510
:1016B0000895089580918B0B90918C0B892B41F4A8
:1016C00081E090E00E94694990938C0B80938B0B92
:1016D00080918B0B90918C0B0895EF92FF920F935A
:1016E0001F93CF93DF93162F072F7A0141155105D2
:1016F00059F4862F0E94C62B31E020E0019709F0B3
:1017000030E0C32FD22F26C04130510509F5262FD6
:10171000663310F02AEC260F80917B00922F987090
:10172000877F892B80937B002770206420937C0027
:1017300080917A00806480937A0080917A0086FD9F
:10174000FCCFC091780080917900D0E0D82B02C006
:10175000C0E0D0E082E0E816F10410F582E095E008
:101760000E94C33C82EA94E00E94C33C88ED94E06E
:101770000E94C33C812F902F0E94363D82EA94E064
:101780000E94C33C8AED94E00E94C33CCE010E94BB
:10179000363D0E94801B0E948A1A80E090E002C0C1
:1017A00081E090E0DF91CF911F910F91FF90EF903A
:1017B00008958091890B90918A0B892BA1F480E781
:1017C00090E00E946949FC01F9969C0123593F4F22
:1017D000DF01D8971C921192E217F307C9F7909393
:1017E0008A0B8093890B8091890B90918A0B0895C5
:1017F00086E095E00E94C33C0E94801B0E94C61DAB
:101800000E94801B0E949C1AD4DF40E050E068E0F8
:1018100070E063DFCEDF40E050E069E070E05DDF64
:10182000C8DF40E050E06AE070E057DFC2DF40E030
:1018300050E06DE070E051DF80E090E008956F923D
:101840007F928F929F92AF92BF92CF92DF92EF9250
:10185000FF920F931F93CF93DF93FB01E2A8F3A8AE
:1018600086A497A4A0A8B1A8C6A0D7A062A073A080
:10187000068D178D9EDFEC019701A301B8017BDC7B
:10188000C501B4010E94292D9701A601B801CE011E
:1018900072DC80E090E0DF91CF911F910F91FF907B
:1018A000EF90DF90CF90BF90AF909F908F907F9000
:1018B0006F9008950F931F93CF93DF93FB0102A9BD
:1018C00013A9C68DD78D75DFA801BE0106DF80E0A4
:1018D00090E0DF91CF911F910F9108951F93CF93C7
:1018E000DF931F92CDB7DEB7FB0162A9168D698326
:1018F00060DF6981812F0E94E22C80E090E00F90F0
:10190000DF91CF911F910895EF92FF920F931F9354
:10191000CF93DF93FB01E2A8F3A802A113A1C68D28
:10192000D78D47DF9701A801BE0125DC80E090E05C
:10193000DF91CF911F910F91FF90EF90089508953F
:101940000895089508950895CF93DF93FC012489A5
:10195000358946895789C28DD38D6089718982897D
:1019600093892031E7E23E074105510529F012161F
:1019700013061406150624F0DE019B01AC0109C014
:101980000E94A55120E43CE940E050E00E94425012
:10199000DE010E946850DF91CF910895FC0181E043
:1019A00090E0958F848F1182108215821482108AA4
:1019B000118A128A138A118E108E80E197E2A0E0BC
:1019C000B0E0848B958BA68BB78B1286108614861D
:1019D00015861686178608958EBD00000DB407FE85
:1019E000FDCF8EB50895CF92DF92EF92FF920F93C5
:1019F0001F93CF93DF93EC0160E086E10E94EE2B12
:101A00008C8D9D8D24E0880F991F2A95E1F78F60BA
:101A1000E3DF83E290E00197F1F704E010E0C12CEE
:101A2000D12C7601FE2CED2CDC2CCC2481E0D4DFF3
:101A3000C82A01501109B1F761E086E10E94EE2B3E
:101A4000C88AD98AEA8AFB8ADF91CF911F910F91C8
:101A5000FF90EF90DF90CF90089508950895089536
:101A60000895089508952F923F924F925F926F923A
:101A70007F928F929F92AF92BF92CF92DF92EF921E
:101A8000FF920F931F93CF93DF93CDB7DEB7E0970D
:101A90000FB6F894DEBF0FBECDBF1C012A013B017B
:101AA0000F83188729873A8728960EAD1FAD289790
:101AB000FC01EF59FD4F60817181828193810E9409
:101AC000164F9B01AC01C301B2010E94754F0E94E9
:101AD0006C516D877E878F87988BF101EB59FD4F95
:101AE00060817181828193810E94164F9B01AC01BC
:101AF0006F81788589859A850E94754F0E946C5107
:101B00006F8B788F898F9A8FF101E759FD4F608134
:101B10007181828193810E94164F9B01AC01C701A4
:101B2000B6010E94754F0E946C516B8F7C8F8D8F18
:101B30009E8F0E94612D6B8B7C8B8D8B9E8BF10118
:101B4000EE51FE4F118210823296118210823E9623
:101B5000A114B10461F0C501A0E0B0E04081518161
:101B60006281738184179507A607B70714F0A080D8
:101B7000B180F101EA50FE4F8114910461F0C4017B
:101B8000A0E0B0E0408151816281738184179507A4
:101B9000A607B70714F080809180F101E650FE4F50
:101BA0000115110561F0C801A0E0B0E0408151814C
:101BB0006281738184179507A607B70714F0008127
:101BC00011819101205F3F4F3A8B298BC501A0E025
:101BD000B0E0F10180A791A7A2A7B3A72101FAE87D
:101BE0004F0E511CA12CB12CD20158968D929D9272
:101BF000AD92BC925B973101BCEF6B1ABEEF7B0AD2
:101C000020E030E0F301008F118F228F338F0E948C
:101C1000801B0E94801B0E94801B0E94801B4091A1
:101C20004C0750914D0760914E0770914F074DA79B
:101C30005EA76FA778AB0E94801B809150079091A0
:101C40005107A0915207B09153078F839887A987B6
:101C5000BA870E94801B8090540790905507A090EF
:101C60005607B0905707F101E359FD4F10821182DA
:101C70001282138234961082118212821382349659
:101C8000108211821282138234961182108232964F
:101C90001182108232961182108232964DA55EA575
:101CA0006FA578A9408351836283738334968F81B3
:101CB0009885A985BA8580839183A283B38334965E
:101CC00080829182A282B3822996EFAC29970D85FA
:101CD0001E852F85388989899A890E9444328823F4
:101CE000F9F088E493E00E94C33C81EB94E00E9409
:101CF000C33CF101EE5AFF4F608171818281938173
:101D0000E15FFD4F20813181428153810E94425029
:101D1000CA01B9010E940F3D0E94801B0E948A1ACD
:101D20002A96EFAC2A970F89188D298D3A8D4F810D
:101D3000588569857A85C2010E9444328823F9F06A
:101D400084E493E00E94C33C81EC94E00E94C33C95
:101D5000F101E453FF4F6081718182819381E756E5
:101D6000FE4F20813181428153810E944250CA013D
:101D7000B9010E940F3D0E94801B0E948A1A2B9677
:101D8000EFAC2B970B8D1C8D2D8D3E8DB501A401D5
:101D9000C3010E9444328823F9F080E493E00E945A
:101DA000C33C81ED94E00E94C33CF101EA5BFE4F2D
:101DB0006081718182819381ED5DFE4F208131814F
:101DC000428153810E944250CA01B9010E940F3DD5
:101DD0000E94801B0E948A1AD10151961C92F10127
:101DE000E557FF4F1082E658FF4F1082C1010E9455
:101DF000901EC1010E94921E89899A890E947F3695
:101E0000C2010E947F36C3010E947F3681E090E0CC
:101E1000F101E751FE4F918380837101B5E1EB1A27
:101E2000BEEFFB0AF70191838083810103511E4FAE
:101E3000D8018D939C9341E050E069897A89C10172
:101E40000E94D81BF70140815181B201C1010E945B
:101E5000D81BD8014D915C91B301C1010E94D81BE0
:101E600011E0F101E253FD4F108389899A890E94A4
:101E70003132C2010E943132C3010E94313264E624
:101E800070E080E090E00E94292DC1018A519E4FB0
:101E9000FC011083D101A951BE4F1C93A1014851EF
:101EA0005E4FFA0110832996FFAD2997F1110FC0FB
:101EB0002A962FAD2A97211105C02B963FAD2B975F
:101EC000332339F1910121593F4FF90110822A96AC
:101ED000FFAD2A97F11105C0910127513F4FF9013C
:101EE00010822B96FFAD2B97F11105C091012D5952
:101EF0003E4FF901108229962FAD2997FC012083CE
:101F00002A963FAD2A973C932B96EFAD2B97DA019B
:101F1000EC9389899A890E94ED33C2010E94ED33C6
:101F2000C3010E94ED3389899A890E944333C2011B
:101F30000E944333C3010E9443330E94801BDC0193
:101F40001C968C918D8718861F82F101EA51FE4FF5
:101F5000F88FEF8B910129513E4F3C8F2B8FA101C0
:101F600048515E4F58A34F8FC10187519E4F9EA38A
:101F70008DA3D101A551BE4FB8A7AFA3EC55F14039
:101F8000FAA3E9A3235E31093CA32BA3FE96FAA78B
:101F9000E9A7225C3F4F3CA72BA7AF89B88D8C9156
:101FA00081110BC0EB8DFC8D8081811106C0AF8D3E
:101FB000B8A18C91882309F459C3BD85B11156C3CA
:101FC000C1010E946E1E4DA15EA169897A89C1017D
:101FD0000E942E1C4FA158A5B201C1010E942E1CC7
:101FE000A10143515E4FB301C1010E942E1C89899A
:101FF0009A890E94AD33C2010E94AD33C3010E9491
:10200000AD33F101EE58FF4F8081882341F189897A
:102010009A890E94ED33F101E755FD4F80818823B5
:10202000D1F0610133E6C31A3DEFD30A710142E4F6
:10203000E41A4DEFF40A810105571D4F9101215813
:102040003D4FA10143595D4FB10162587E4F8989CF
:102050009A890E940E30F101EE58FF4F1082F10173
:10206000E451FF4F8081882331F1C2010E94ED339A
:10207000F101E655FD4F80818823C9F061015FE5DC
:10208000C51A5DEFD50A710180E4E81A8DEFF80AF0
:10209000810101571D4F91012D573D4FA1014F580F
:1020A0005D4FB10164567E4FC2010E940E30F101B6
:1020B000E451FF4F1082F101EA59FE4F80818823DD
:1020C00031F1C3010E94ED33F101E555FD4F8081EF
:1020D0008823C9F061019BE5C91A9DEFD90A7101F6
:1020E000AEE3EA1AADEFFA0A81010D561D4F9101D8
:1020F00029573D4FA1014B585D4FB10166547E4FAA
:10210000C3010E940E30F101EA59FE4F1082810195
:1021100001591F4FF80180818823E9F1E85DFD4FE7
:1021200060817181072E000C880B990B0E94164F5D
:102130009B01AC01F101E359FD4F60817181828106
:1021400093810E949D51181634F5D8011C9266E2C5
:1021500074E0810108521E4FC8010E94102B6BE4ED
:1021600075E0C8010E94102B6EE973E0C8010E945F
:10217000102B2996BFAD2997BB2309F471C3C10168
:1021800082589E4F0E940A3EF101E25BFF4F10828F
:10219000118212821382810107511F4FD8018C9145
:1021A000882309F43EC0F101E756FD4F608171813B
:1021B000072E000C880B990B0E94164F9B01AC0157
:1021C000F101EF58FD4F60817181828193810E94FE
:1021D0009D51181634F5D8011C9266E274E0810115
:1021E00008521E4FC8010E94102B63E775E0C8011A
:1021F0000E94102B6EE973E0C8010E94102B2A96F2
:10220000BFAD2A97BB2309F430C3C10184569E4F4A
:102210000E940A3EE9A1FAA1FE9610821182128262
:10222000138281010D591E4FF80180818823E9F145
:10223000E85CFE4F60817181072E000C880B990BC2
:102240000E94164F9B01AC01F101EB58FD4F6081DC
:102250007181828193810E949D51181634F5D801B5
:102260001C9266E274E0810108521E4FC8010E9470
:10227000102B6BE975E0C8010E94102B6EE973E02A
:10228000C8010E94102B2B96BFAD2B97BB2309F4DE
:10229000F1C2C10186549E4F0E940A3EEBA1FCA1EF
:1022A000FE96108211821282138260E089899A89D7
:1022B0000E94BC32882361F0F101E25BFF4F108283
:1022C000118212821382C10182589E4F0E940A3EDF
:1022D00060E0C2010E94BC32882361F0A9A5BAA5C2
:1022E0001D921D921D921C921397C10184569E4F00
:1022F0000E940A3E60E0C3010E94BC32882359F06C
:10230000EBA5FCA51082118212821382C1018654B2
:102310009E4F0E940A3EF101E159FF4F8081AF8933
:10232000B88D8C93E658FF4F8081EB8DFC8D8083B8
:10233000F101ED59FE4F8081AF8DB8A18C93E5512D
:10234000F1404081518162817381E9A1FAA1FE9639
:1023500080809180A280B380EBA1FCA1FE96C0801A
:10236000D180E280F3804DA75EA76FA778AB0E9473
:10237000801B4DA55EA56FA578A940934C0750938F
:102380004D0760934E0770934F070E94801B809209
:10239000500790925107A0925207B09253070E94A3
:1023A000801BC0925407D0925507E0925607F092D6
:1023B0005707C1010E94901EEF89F88D8081882304
:1023C00009F44AC00E94612D2B893C894D895E89A0
:1023D000621773078407950760F40E94612D2B89AB
:1023E0003C894D895E896217730784079507A0F5BC
:1023F0001EC00E94612D6B017C012B893C894D8997
:102400005E89C21AD30AE40AF50AF101EB5AFD4FBC
:102410002081318142815381A8EEB3E00E945E5059
:102420006C157D058E059F0508F429C2D6CF0E9444
:10243000612D6B017C01F101EB5AFD4F208131814F
:1024400042815381A8EEB3E00E945E506C157D0579
:102450008E059F0508F413C2AB8DBC8D8C9188232B
:1024600009F44AC00E94612D2B893C894D895E89FF
:10247000621773078407950760F40E94612D2B890A
:102480003C894D895E896217730784079507A0F51B
:102490001EC00E94612D6B017C012B893C894D89F6
:1024A0005E89C21AD30AE40AF50AF101E75AFD4F20
:1024B0002081318142815381A8EEB3E00E945E50B9
:1024C0006C157D058E059F0508F4F0C1D6CF0E94DE
:1024D000612D6B017C01F101E75AFD4F20813181B3
:1024E00042815381A8EEB3E00E945E506C157D05D9
:1024F0008E059F0508F4DAC1AF8DB8A18C918823B1
:1025000009F44AC00E94612D2B893C894D895E895E
:10251000621773078407950760F40E94612D2B8969
:102520003C894D895E896217730784079507A0F57A
:102530001EC00E94612D6B017C012B893C894D8955
:102540005E89C21AD30AE40AF50AF101E35AFD4F83
:102550002081318142815381A8EEB3E00E945E5018
:102560006C157D058E059F0508F4B7C1D6CF0E9476
:10257000612D6B017C01F101E35AFD4F2081318116
:1025800042815381A8EEB3E00E945E506C157D0538
:102590008E059F0508F4A1C18BEA9BE00E946C2880
:1025A0001816190684F58BEA9BE00E944A288F7D55
:1025B0008534910541F56DE075E0C10188529E4F6B
:1025C0000E94102B84E693E00E94C33C0E94801B73
:1025D000A1D7F101E159FF4F1082E658FF4F108259
:1025E000E658FF4F1082AF89B88D1C92EB8DFC8DA1
:1025F0001082AF8DB8A11C92B1E0BD87E1E0F0E0A0
:10260000F887EF8304C02F813885232B81F062E2A5
:1026100075E0C10188529E4F0E94102BAF89B88D82
:102620001C92EB8DFC8D1082AF8DB8A11C92C10164
:102630000E94793CF101EC51FE4F8081918101961D
:10264000918380838D3291400CF4A7CCD101A452A8
:10265000BE4F8D919C911197892B09F09ECC1496B9
:102660008D919C91892B09F44FC197CC8101045223
:102670001E4FF80180819181892B21F0C1010E94B8
:10268000793CF7CF82E395E00E94C33C2996FFADE9
:102690002997FF2301F12F813885232BE1F43D8514
:1026A00031113EC080E393E00E94C33C0E94801B36
:1026B00031D72A964FAD2A97442369F18CE293E0F3
:1026C0000E94C33C0E94801B25D72B965FAD2B97A1
:1026D00051111AC025C02A968FAD2A97882341F040
:1026E000AF81B885AB2B21F4BD85B11119C0E6CF00
:1026F0002B96EFAD2B97EE2399F02F813885232B66
:1027000079F43D8531110CC088E293E00E94C33C0E
:10271000F7D700D705C02B969FAD2B979111F4CF1B
:10272000810107511E4F85E090E0D8018D939C9365
:102730006101B5E1CB1ABEEFDB0AF601918380831C
:102740007101F3E1EF1AFEEFFF0AD7018D939C931D
:1027500045E050E069897A89C1010E94D81BF601E1
:1027600040815181B201C1010E94D81BD7014D9116
:102770005C91B301C1010E94D81BC1010E94941E4B
:10278000F101E25BFF4F4081518162817381E65824
:10279000FF4F80809180A280B380E658FF4F8081F8
:1027A0009181A281B3818B8B9C8BAD8BBE8B4DA70E
:1027B0005EA76FA778ABA4D74DA55EA56FA578A936
:1027C00040934C0750934D0760934E0770934F070B
:1027D00097D78092500790925107A0925207B092DB
:1027E00053078ED72B893C894D895E8920935407E6
:1027F000309355074093560750935707C1010E94E5
:10280000901EC1010E94921E7BD7D7D6C1010E94A3
:10281000661CD8011D921C92F60111821082D7010C
:102820001D921C9240E050E069897A89C101C0D7AD
:10283000F60140815181B201C101BAD7D7014D9152
:102840005C91B301C101B4D7C1010E94941EBD8542
:10285000BB2309F424C254D721E0FC0124871FC202
:10286000E1E0F0E0F887EF8396CCE1E0F0E0F88774
:10287000EF83D7CCE1E0F0E0F887EF8316CD6CE38F
:1028800073E0810108521E4FC8010E94102B6EE9AF
:1028900073E0C8010E94102B63EC75E0C8010E9430
:1028A000102B22E030E038872F83D6CD68E373E029
:1028B000810108521E4FC8010E94102B6EE973E07F
:1028C000C8010E94102B68ED75E0C8010E94102B12
:1028D00042E050E058874F830FCE64E373E08101FC
:1028E00008521E4FC8010E94102B6EE973E0C80108
:1028F0000E94102B6DEE75E0C8010E94102B82E043
:1029000090E098878F8348CE11821082F101EE51BA
:10291000FE4F80819181009749F460E673E0810168
:1029200008521E4FC8010E94102B96C1019709F052
:10293000A2C1E6D68C01FC0180819181A281B38184
:10294000181619061A061B0644F081E090E0A0E074
:10295000B0E080839183A283B383F8018481958161
:10296000A681B781181619061A061B0644F081E0E5
:1029700090E0A0E0B0E084839583A683B783F8015C
:1029800080859185A285B385181619061A061B063F
:1029900044F081E090E0A0E0B0E080879187A287DA
:1029A000B38760EA73E0CE0101960E94532B6EE27A
:1029B00075E0CE0101960E94102B61EB74E0CE0110
:1029C00001960E94102B60914C0770914D078091E9
:1029D0004E0790914F070E94164F6B017C01D80162
:1029E0006D917D918D919C910E94164F9B01AC0140
:1029F000C701B6010E940451AB01BC01CE01019692
:102A00000E94802A61EC74E0CE0101960E94102B96
:102A10006091500770915107809152079091530730
:102A20000E94164F6B017C01F801648175818681DB
:102A300097810E94164F9B01AC01C701B6010E940D
:102A40000451AB01BC01CE0101960E94802A61EDC8
:102A500074E0CE0101960E94102B60915407709192
:102A6000550780915607909157070E94164F6B01AA
:102A70007C01D80118966D917D918D919C911B9749
:102A80000E94164F9B01AC01C701B6010E94045180
:102A9000AB01BC01CE0101960E94802ABE016F5F8E
:102AA0007F4F810108521E4FC8010E941E2BCE018C
:102AB00001960E944E2B24D6BC01CE0101960AD568
:102AC000BE016F5F7F4FC8010E941E2BCE01019691
:102AD0000E944E2B64E273E0C8010E94102B61EB50
:102AE00074E0C8010E94102BF101E258FE4FFC87F0
:102AF000EB87CF010E94A40C0E94164F6B017C0152
:102B0000F101EF59FD4F60817181828193810E94B3
:102B1000164F9B01AC01C701B6010E940451AB01E5
:102B2000BC01C8010E94B02A61EC74E0C8010E9497
:102B3000102B6101F4E6CF1AFEEFDF0AC6010E94F6
:102B4000A40C0E94164F4B015C01F101EB59FD4FA3
:102B500060817181828193810E94164F9B01AC013B
:102B6000C501B4010E940451AB01BC01C8010E941F
:102B7000B02A61ED74E0C8010E94102B710126E4B7
:102B8000E21A2EEFF20AC7010E94A40C0E94164F0F
:102B90004B015C01F101E759FD4F60817181828138
:102BA00093810E94164F9B01AC01C501B4010E94A4
:102BB0000451AB01BC01C8010E94B02AA1D5BC01DF
:102BC000CE01019687D4BE016F5F7F4FC8010E947E
:102BD0001E2BCE0101960E944E2B60E273E0C801CD
:102BE0000E94102B61EB74E0C8010E94102BEB8552
:102BF000FC85A28DB38D20893189428953890E9439
:102C00006850AB01BC01C8010E94E02A61EC74E08D
:102C1000C8010E94102BF601A28DB38D2089318945
:102C2000428953890E946850AB01BC01C8010E94CF
:102C3000E02A61ED74E0C8010E94102BF701A28D1B
:102C4000B38D20893189428953890E946850AB0134
:102C5000BC01C8010E94E02A53D5BC01CE010196F7
:102C600039D4BE016F5F7F4FC8010E941E2BCE0179
:102C700001960E944E2BF101EE51FE4F8081918111
:102C80000196823091051CF49183808302C01182E9
:102C90001082F101E052FE4F118210827EC980E461
:102CA00095E00E94C33C8F8198850E94363D8EE955
:102CB00093E00E94C33C24D52F8138853093470789
:102CC00020934607C901E0960FB6F894DEBF0FBE09
:102CD000CDBFDF91CF911F910F91FF90EF90DF90CB
:102CE000CF90BF90AF909F908F907F906F905F90AC
:102CF0004F903F902F900895662319F08FEA93E04C
:102D000002C088EA93E00C94C33C0C94FE490C94F6
:102D1000FE49AF92BF92CF92DF92EF92FF920F9354
:102D20001F93CF93DF93EC018AE190E09E8B8D8B14
:102D30008BE190E0988F8F8B89E190E09A8F898F5B
:102D40008FE090E09C8F8B8F8EE190E09E8F8D8F37
:102D50008EE090E098A38F8F85E490E09AA389A3FA
:102D600084E490E09CA38BA3FE01E657FF4F80E232
:102D700090E09683858381E290E0908787838FE15E
:102D800090E0928781871486138616861586108AAE
:102D9000178683E490E0928B818B82E490E0948BA1
:102DA000838BE658FF4F83E290E09683858384E22D
:102DB00090E09087878382E290E0928781871486F3
:102DC000138616861586108A178681E490E0928B0A
:102DD000818B80E490E0948B838BEB51FF4F1182C9
:102DE0001082329611821082329611821082CE01A8
:102DF0000E94AF20CE01C6D7CE0182589E4F41E03F
:102E000050E0FC01558F448FDE01A456BE4F24E0F4
:102E100030E05D963C932E935C975E01F6E4AF1A2A
:102E2000FEEFBF0A28E030E0F501358F248F20E166
:102E300030E0FC013183208321E130E035832483BD
:102E40002FEF3FEF338322833783268362856087AA
:102E50006385618767E170E011967C936E9368E10A
:102E600070E015967C936E93149713963C932E9373
:102E7000129717963C932E9316971A966C911A9761
:102E800018966C9318971B966C911B9719966C93D8
:102E900019976DE170E0F501718360836CE170E07A
:102EA00075836483338322833783268362856087B7
:102EB00063856187BE016C537D4FFB016081718129
:102EC0008E010E541D4FF801C080D180E280F38046
:102ED00006501109F80100811181FC01118F008F4A
:102EE000C48AD58AE68AF78A6130710519F4338F6E
:102EF000228F03C0FC01538F428FCE018A539D4F16
:102F0000FC01808191819E012A543D4FF90140814D
:102F100051816281738128503109F9012081318109
:102F200059963C932E93589754964D935D936D9379
:102F30007C935797019719F48FEF9FEF02C081E0C0
:102F400090E05B969C938E935A97DE01A853BD4FF9
:102F50008D919C9111971E974D915D916D917C91F2
:102F6000C055DD4F28813981F501318F208F448B89
:102F7000558B668B778B019719F48FEF9FEF03C00A
:102F800081E090E0F501938F828FDF91CF911F91C7
:102F90000F91FF90EF90DF90CF90BF90AF9008958A
:102FA0002F923F924F925F926F927F928F929F9259
:102FB000AF92BF92CF92DF92EF92FF920F931F9347
:102FC000CF93DF93CDB7DEB7CA57D1090FB6F894C8
:102FD000DEBF0FBECDBF8C01FC01108211821282B8
:102FE0001382148215821682178210861186128629
:102FF000138614861586168617862C01F0E14F0E6F
:10300000511CC2010E94A13668018AE8C80ED11C79
:10301000C6010E94A1367801ECEFEE1AEEEFFE0A2F
:10302000C7010E94A1363801F2E86F1AFEEF7F0A4D
:10303000C3010E94CE0C480184E6881A8EEF980ADC
:10304000C4010E94CE0C5801E6E4AE1AEEEFBE0AAF
:10305000C5010E94CE0C60EA73E0C80188529E4F01
:103060000E94532BF801E252FE4F118210823296D9
:103070001182108232961182108232961182108251
:1030800032961082319610823196108231961182DA
:1030900010823296118210823296118210823296FC
:1030A00010823196108231961082319610821182F0
:1030B0001282138234961082118212821382349605
:1030C000108211821282138234961082118212822F
:1030D00013823496108211821282138234961082E7
:1030E000118212821382349610821182128213820C
:1030F00034961082118212821382349610821182C9
:1031000012821382349610821182128213823496B4
:1031100010821182128213823496108211821282DE
:103120001382349610821182128213823496108296
:1031300011821282138234961082118212821382BB
:103140003496108231961082319610823196108218
:10315000118212821382349610821182128213829B
:103160003496108211821282138234961082319624
:1031700010823196108231961082319610823196EB
:1031800010823196108231961082319610823196DB
:1031900010823196108231961082319610823196CB
:1031A00010823196108231961082319610823196BB
:1031B00010823196108231961082319610823196AB
:1031C00010823196108231961082319610821182CF
:1031D00012821382349610821182128213823496E4
:1031E0001082118212821382D801AF59BD4F8CE038
:1031F000ECE4F3E001900D928A95E1F7F801E359D0
:10320000FD4F108211821282138234961082118235
:1032100012821382349610821182128213823496A3
:10322000118210823296118210823296118210829F
:103230003296108211821282138234961082118289
:103240001282138234961082118212821382349673
:10325000108211821282138234961082118212829D
:103260001382349610821182128213823496118254
:10327000108232961182108232961182108232961A
:10328000108211821282138234961082118212826D
:103290001382349610821182128213823496108225
:1032A00031961082319610823196118210823296B8
:1032B000118210823296118210823296108211820F
:1032C00012821382349610821182128213823496F3
:1032D00010821182128213823496118210823296E9
:1032E00011821082329611821082329611821082DF
:1032F0003296118210823296118210823296118299
:1033000010823296118210821801F2E32F1AFDEF1B
:103310003F0AF1011082CE0101960E94A1368AE790
:10332000FE013196D20101900D928A95E1F7CE010E
:1033300001960E94A1368AE7FE013196D6010190DE
:103340000D928A95E1F7CE0101960E94A1368AE797
:10335000FE013196D70101900D928A95E1F788E53B
:10336000F801808B89E5F60180838AE5F701808387
:10337000CE0101960E94CE0C8EE1FE013196D30162
:1033800001900D928A95E1F7CE0101960E94CE0C34
:103390008EE1FE013196D40101900D928A95E1F7FC
:1033A000CE0101960E94CE0C8EE1FE013196D50130
:1033B00001900D928A95E1F7C801ABDCF101108212
:1033C000C658DF4F0FB6F894DEBF0FBECDBFDF91FA
:1033D000CF911F910F91FF90EF90DF90CF90BF9012
:1033E000AF909F908F907F906F905F904F903F90A5
:1033F0002F900895CF93DF9380919C0B90919D0B1C
:10340000892B51F48FEC92E00E946949EC01C8DDF0
:10341000D0939D0BC0939C0B80919C0B90919D0B26
:10342000DF91CF9108954F925F926F927F928F922A
:103430009F92AF92BF92CF92DF92EF92FF920F9343
:103440001F93CF93DF9300D01F92CDB7DEB7FB0160
:103450001689078982889388A684B784C284D38416
:10346000E484F5844680578060847184428153816E
:103470006481758149835A836B837C83BBDF1F9290
:103480001F921F920F931F939301820149815A81CA
:103490006B817C810E94330D0F900F900F900F90E5
:1034A0000F9080E090E00F900F900F900F90DF91C1
:1034B000CF911F910F91FF90EF90DF90CF90BF9031
:1034C000AF909F908F907F906F905F904F900895F6
:1034D00008950895CF93DF93EC0160EA73E00E94B2
:1034E000532B62E076E0CE010E94102B40914807FA
:1034F0005091490760914A0770914B07CE010E9495
:10350000E02A6EE973E0CE010E94102BCE01DF911C
:10351000CF91089582E096E00E94C33C60914807F5
:103520007091490780914A0790914B070E940F3D87
:103530008EE993E00C94C33C0F931F93CF93DF93DA
:10354000EC0185E096E00E94C33C89E096E00E9491
:10355000C33C06E91BE0F8016081CE01CDDB8DE0C4
:1035600096E00E94C33CF8016181CE01C5DB81E198
:1035700096E00E94C33CF8016281CE01BDDB85E18B
:1035800096E00E94C33CF8016381CE01B5DB89E17E
:1035900096E00E94C33CF8016481CE01ADDB8DE171
:1035A00096E00E94C33CF8016581CE01A5DBCE0107
:1035B000DF91CF911F910F91ADCFCF92DF92EF921C
:1035C000FF92CF93DF93EC0188819981AA81BB811F
:1035D000181619061A061B0644F081E090E0A0E0D8
:1035E000B0E088839983AA83BB838C819D81AE815F
:1035F000BF81181619061A061B0644F081E090E0F8
:10360000A0E0B0E08C839D83AE83BF8388859985DD
:10361000AA85BB85181619061A061B0644F081E018
:1036200090E0A0E0B0E088879987AA87BB878EE208
:1036300095E00E94C33C81EB94E00E94C33C609102
:103640004C0770914D0780914E0790914F070E9453
:10365000164F6B017C01688179818A819B810E9470
:10366000164F9B01AC01C701B6010E94045142E014
:103670000E943B3D81EC94E00E94C33C6091500766
:103680007091510780915207909153070E94164FF5
:103690006B017C016C817D818E819F810E94164F20
:1036A0009B01AC01C701B6010E94045142E00E9497
:1036B0003B3D81ED94E00E94C33C609154077091C2
:1036C000550780915607909157070E94164F6B013E
:1036D0007C01688579858A859B850E94164F9B01B0
:1036E000AC01C701B6010E94045142E00E943B3D7B
:1036F000CE01DF91CF91FF90EF90DF90CF900ACF76
:103700008091940B9091950B892B91F58DE090E031
:103710000E946949FC01148610924C0710924D07D3
:1037200010924E0710924F071092500710925107B7
:103730001092520710925307109254071092550797
:1037400010925607109257071092930B1092920BFB
:10375000109248071092490710924A0710924B079F
:1037600010924707109246079093950B8093940B05
:103770008091940B9091950B08950F931F93CF9385
:10378000DF938B01EA018CE593E00E94C33C82EA5F
:1037900094E00E94C33CF80180810E94043DCE0168
:1037A0000E94363DADDFDF91CF911F910F91B2CED8
:1037B000CF92DF92EF92FF920F931F93CF93DF93FD
:1037C000CDB7DEB728970FB6F894DEBF0FBECDBFDA
:1037D0008B016A0188529E4F7C0168E573E00E946C
:1037E000102B62EA74E0C7010E94102BF80180815F
:1037F00089831A8241E050E08E010F5F1F4FB801AC
:10380000C7010E94532A4AE0B801C6010E94C34A78
:10381000F80101900020E9F73197AF01401B510BEF
:10382000B801C7010E94532A6BDFBC01C80152DEF8
:10383000B801C7010E941E2BC8010E944E2B28967A
:103840000FB6F894DEBF0FBECDBFDF91CF911F91B1
:103850000F91FF90EF90DF90CF900895FC01DB0176
:10386000AD59BF4F8C91882319F022E030E002C09F
:1038700020E030E0DB01AB59BF4F8C91882311F081
:1038800023E030E0DB01AC59BF4F8C91882311F06D
:1038900024E030E0DB01AA59BF4F8C91882311F05E
:1038A00026E030E0DA018D919C918217930721F098
:1038B00091E0121613060CF090E0DA012D933C9380
:1038C000992319F0A901CF0173CF08958F929F9288
:1038D000AF92BF92CF92DF92EF92FF920F931F931E
:1038E000CF93DF93EC0184E293E00E94C33C81EB31
:1038F00094E00E94C33C6E0182E8C81A8EEFD80A99
:10390000C6010E94A40C0E94164F4B015C01FE01EF
:10391000EF59FD4F60817181828193810E94164F22
:103920009B01AC01C501B4010E94045142E00E9418
:103930003B3D81EC94E00E94C33C7E01E4E6EE1A3C
:10394000EEEFFE0AC7010E94A40C0E94164F4B0125
:103950005C01FE01EB59FD4F608171818281938191
:103960000E94164F9B01AC01C501B4010E94045195
:1039700042E00E943B3D81ED94E00E94C33C8E01F9
:1039800006541E4FC8010E94A40C0E94164F4B0102
:103990005C01C759DD4F688179818A819B810E94D2
:1039A000164F9B01AC01C501B4010E94045142E0D5
:1039B0000E943B3DA5DEAEDD80E293E00E94C33C69
:1039C00081EB94E00E94C33CF601A28DB38D208967
:1039D0003189428953890E9468500E940F3D81ECD1
:1039E00094E00E94C33CF701A28DB38D20893189F8
:1039F000428953890E9468500E940F3D81ED94E0F6
:103A00000E94C33CF801A28DB38D2089318942897F
:103A100053890E9468500E940F3D72DEDF91CF9162
:103A20001F910F91FF90EF90DF90CF90BF90AF90DC
:103A30009F908F906FCD4F925F926F927F928F92F7
:103A40009F92AF92BF92CF92DF92EF92FF920F932D
:103A50001F93CF93DF9300D01F92CDB7DEB70E94A4
:103A6000560A40903408509035086090360870909F
:103A700037080E94560A8090380890903908A09024
:103A80003A08B0903B083CDEC0904C07D0904D0700
:103A9000E0904E07F0904F0733DEC701B6010E9459
:103AA000164F6B017C01C301B2010E94164F9B01AE
:103AB000AC01C701B6010E9404512B013C01609189
:103AC00050077091510780915207909153070E94BF
:103AD000164F6B017C01C501B4010E94164F9B017A
:103AE000AC01C701B6010E940451AB01BC0149837E
:103AF0005A836B837C837EDC1F921F921F921F92DE
:103B00001F92812C912CA12CB12CC12CD12C76018F
:103B100049815A816B817C818A019B01B301A20199
:103B20000E94330D67DC1F921F921F921F921F92FB
:103B300097018601B301A2010E94330D5BDC1F9245
:103B40001F921F921F921F9297018601B701A60133
:103B50000E94330D0FB6F894DEBF0FBECDBF80E0DC
:103B600090E00F900F900F900F90DF91CF911F91E9
:103B70000F91FF90EF90DF90CF90BF90AF909F900C
:103B80008F907F906F905F904F900895CF93DF93C9
:103B900085E40E94C62BEC01B3DD91E0CD2B09F446
:103BA00090E09093960B84E40E94C62BEC01A8DD74
:103BB00091E0CD2B09F490E09093970B83E40E9461
:103BC000C62BEC019DDD91E0CD2B09F490E09093A4
:103BD000980B82E40E94C62BEC0192DD91E0CD2B84
:103BE00009F490E09093990B81E40E94C62BEC01BC
:103BF00087DD91E0CD2B09F490E090939A0B80E45F
:103C00000E94C62BEC017CDD91E0CD2B09F490E005
:103C100090939B0BDF91CF910895CF93DF93EC01AD
:103C20002AEC30E04BEC50E069EC70E00E94BF2FD2
:103C30002EEC30E04FEC50E06DEC70E0CE010C96D5
:103C40000E94BF2F24ED30E045ED50E063ED70E0C1
:103C5000CE0148960E94BF2F28ED30E049ED50E09C
:103C600067ED70E0CE0184960E94BF2F2EED30E00C
:103C70004FED50E06DED70E0CE01C096DF91CF9139
:103C80000C94BF2FCF93DF938091900B9091910B69
:103C9000892BE9F48CE390E00E946949EC01FC0176
:103CA000CC96118210823C96E817F907D1F7198259
:103CB00018821D861C86198E188E1DA21CA219AA98
:103CC00018AACE01AADFD093910BC093900B8091DC
:103CD000900B9091910BDF91CF910895CF93DF934B
:103CE000EC0183B183B1E0E0F1E080818081CE011D
:103CF00082589E4F0E94F30C83B183B180B180B192
:103D0000CE0184569E4F0E94F30C83B183B180B1E3
:103D100080B1CE0186549E4FDF91CF910C94F30C6D
:103D2000EFDC34CFEDDC08CCCF93DF93EC01FC016A
:103D3000E253FD4F1082EE58F1098081811104C0D9
:103D4000CE0140960E941F32FE01EF5BFD4F808145
:103D5000811105C0CE0186579F4F0E941F32FE0180
:103D6000EE5BFD4F8081811105C0CE018C5F9E4FBF
:103D70000E941F3264E670E080E090E0DF91CF9116
:103D80000C94292D2F923F924F925F926F927F92C7
:103D90008F929F92AF92BF92CF92DF92EF92FF925B
:103DA0000F931F93CF93DF93EC010E94560AFE01FD
:103DB000E956FD4F809114099091150991838083F4
:103DC0000E94560AFE01E756FD4F80911809909116
:103DD0001909918380830E94560AFE01E556FD4F22
:103DE00080911C0990911D09918380830E94560A3D
:103DF0008E0103561D4F60913C0970913D098091E1
:103E00003E0990913F090E94164FF801608371832B
:103E1000828393830E94560A1E01FFE52F1AFDEF4D
:103E20003F0A609140097091410980914209909147
:103E300043090E94164FF10160837183828393834B
:103E40000E94560A20E030E048EC52E4F80160811C
:103E50007181828193810E9404512B013C0120E0F9
:103E600030E048EC52E4F1016081718182819381FC
:103E70000E9404514B015C01609144097091450915
:103E800080914609909147090E94164F20E030E04A
:103E900048EC52E40E9404516B017C012AE037EDAA
:103EA00043E25CE3C301B2010E949D5118168CF4F9
:103EB00020E030E046EC52E4C301B2010E94104F12
:103EC00087FD0FC0412C512C46EC642E42E4742E29
:103ED00008C05AE0452E57ED552E53E2652E5CE39F
:103EE000752EF80140825182628273822AE037ED9A
:103EF00043E25CE3C501B4010E949D5118168CF4A5
:103F000020E030E046EC52E4C501B4010E94104FBD
:103F100087FD0FC0812C912C26ECA22E22E4B22E1C
:103F200008C03AE0832E37ED932E33E2A32E3CE314
:103F3000B32EF10180829182A282B3822AE037ED12
:103F400043E25CE3C701B6010E949D5118168CF450
:103F500020E030E046EC52E4C701B6010E94104F69
:103F600087FD0FC0C12CD12C86ECE82E82E4F82E00
:103F700008C09AE0C92E97EDD92E93E2E92E9CE372
:103F8000F92EFE01EB55FD4FC082D182E282F38211
:103F90000E94560A8091FC089091FD08FE01E455AC
:103FA000FD4F918380830E94560A80910009909171
:103FB0000109FE01E255FD4F918380830E94560A5C
:103FC0008091040990910509FE01E055FD4F918310
:103FD00080830E94560A8091240990912509A0911E
:103FE0002609B0912709FE01EE54FD4F808391838D
:103FF000A283B3830E94560A8091280990912909CF
:10400000A0912A09B0912B09FE01EA54FD4F80834B
:104010009183A283B3830E94560A80912C099091C8
:104020002D09A0912E09B0912F09FE01E654FD4FF4
:1040300080839183A283B3830E94560A80914C09A6
:1040400090914D09FE01E254FD4F918380830E94BF
:10405000560A8091500990915109FE01E054FD4F9C
:10406000918380830E94560A80915409909155094A
:10407000FE01EE53FD4F918380830E94560A80918A
:10408000640990916509FE01EC53FD4F9183808393
:104090000E94560A8091680990916909FE01EA53CD
:1040A000FD4F918380830E94560A80916C09909104
:1040B0006D09FE01E853FD4F918380830E94560AEB
:1040C0008091EC089091ED08A091EE08B091EF0876
:1040D000FE01E755FD4F0197A105B10519F481E0F7
:1040E000808301C010820E94560A8091F00890914E
:1040F000F108A091F208B091F308FE01E655FD4FDA
:104100000197A105B10519F481E0808301C01082F7
:104110000E94560A8091F4089091F508A091F60843
:10412000B091F708C555DD4F0197A105B10519F408
:1041300081E0888301C01882DF91CF911F910F9198
:10414000FF90EF90DF90CF90BF90AF909F908F90B7
:104150007F906F905F904F903F902F9008952F9297
:104160003F924F925F926F927F928F929F92AF9207
:10417000BF92CF92DF92EF92FF920F931F93CF9354
:10418000DF93CDB7DEB760970FB6F894DEBF0FBEF2
:10419000CDBF988B8F870E94560AEF85F889E15131
:1041A000FE4F81E040912408509125086091260837
:1041B00070912708452B462B472B09F480E080831C
:1041C0000E94560AEF85F889E051FE4F81E0409148
:1041D00028085091290860912A0870912B08452BD6
:1041E000462B472B09F480E080830E94560AEF8516
:1041F000F889EF50FE4F81E040912C0850912D0836
:1042000060912E0870912F08452B462B472B09F4FF
:1042100080E080830E94560A80917408909175080E
:10422000A0917608B0917708EF85F889EE50FE4F9F
:1042300080839183A283B3830E94560A8091780879
:1042400090917908A0917A08B0917B08EF85F88960
:10425000EA50FE4F80839183A283B3830E94560A63
:1042600080917C0890917D08A0917E08B0917F0894
:10427000EF85F889E650FE4F80839183A283B38354
:104280000E94560A80914C0890914D08A0914E08CA
:10429000B0914F08EF85F889E65FFD4F80839183E9
:1042A000A283B3830E94560A8091500890915108CE
:1042B000A0915208B0915308EF85F889E25FFD4F55
:1042C00080839183A283B3830E94560A809154080D
:1042D00090915508A0915608B0915708EF85F8893C
:1042E000EE5EFD4F80839183A283B3830E94560AC2
:1042F00080915C0890915D08A0915E08B0915F0884
:10430000EF85F889EA5EFD4F80839183A283B383B2
:104310000E94560A8091600890916108A0916208FD
:10432000B0916308EF85F889E65EFD4F8083918345
:10433000A283B3830E94560A809164089091650815
:10434000A0916608B0916708EF85F889E25EFD4F9D
:1043500080839183A283B3830E94560A8091FC07D5
:104360009091FD07A091FE07B091FF07EF85F889B6
:10437000EE5DFD4F80839183A283B3830E94560A32
:104380008091000890910108A0910208B091030863
:10439000EF85F889EA5DFD4F80839183A283B38323
:1043A0000E94560A8091040890910508A091060881
:1043B000B0910708EF85F889E65DFD4F8083918312
:1043C000A283B3830E94560AEF85F889E25DFD4F10
:1043D00081E02091D4073091D5072130310509F0D3
:1043E00080E080830E94560AEF85F889E15DFD4FE9
:1043F00081E02091D8073091D9072130310509F0AB
:1044000080E080830E94560AEF85F889E05DFD4FC9
:1044100081E02091DC073091DD072130310509F082
:1044200080E080830E94560AEF85F889E45BFD4FA7
:1044300081E04091AC075091AD076091AE0770915B
:10444000AF07452B462B472B09F480E080830E9461
:10445000560AEF85F889E35BFD4F81E04091B00794
:104460005091B1076091B2077091B307452B462B6D
:10447000472B09F480E080830E94560AEF85F88973
:10448000E25BFD4F81E04091B4075091B507609128
:10449000B6077091B707452B462B472B09F480E0F0
:1044A00080830E94560AEF85F889E15BFD4F81E029
:1044B0004091840850918508609186087091870822
:1044C000452B462B472B09F480E080830E94560A37
:1044D000EF85F889E05BFD4F81E0409188085091BD
:1044E000890860918A0870918B08452B462B472BD1
:1044F00009F480E080830E94560AEF85F889EF5A1C
:10450000FD4F81E040918C0850918D0860918E089C
:1045100070918F08452B462B472B09F480E0808350
:104520000E94560AEF85F889EE5AFD4F81E02091EE
:10453000BC073091BD072130310509F080E0808350
:104540000E94560AEF85F889ED5AFD4F81E02091CF
:10455000C0073091C1072130310509F080E0808328
:104560000E94560AEF85F889EC5AFD4F81E02091B0
:10457000C4073091C5072130310509F080E0808300
:104580000E94560A8091840790918507A091860722
:10459000B0918707EF85F889EB5AFD4F80839183AF
:1045A000A283B3830E94560A80918807909189075D
:1045B000A0918A07B0918B07EF85F889E75AFD4FE4
:1045C00080839183A283B3830E94560A80918C07D3
:1045D00090918D07A0918E07B0918F07EF85F88994
:1045E000E35AFD4F80839183A283B3830E94560ACE
:1045F000EF85F889E05CFD4F81E040919407509190
:1046000095076091960770919707452B462B472B8E
:1046100009F480E080830E94560AEF85F889EF5BF9
:10462000FD4F81E0409198075091990760919A075A
:1046300070919B07452B462B472B09F480E0808324
:104640000E94560AEF85F889EE5BFD4F81E04091AC
:104650009C0750919D0760919E0770919F07452B85
:10466000462B472B09F480E080830E94560A8091F4
:104670008C0990918D09A0918E09B0918F09EF85D9
:10468000F889EF5CFD4F80839183A283B3830E94FE
:10469000560A8091900990919109A0919209B09148
:1046A0009309EF85F889EB5CFD4F80839183A283AA
:1046B000B3830E94560A8091940990919509A09124
:1046C0009609B0919709EF85F889E75CFD4F8083E3
:1046D0009183A283B3830E94560AEF85F889ED5B2C
:1046E000FD4F81E02091EC073091ED07213031053D
:1046F00009F080E08083EF85F889EC5BFD4F108244
:10470000EF85F889EB5BFD4F10820E94560AEF851A
:10471000F889EA5BFD4F81E02091E8073091E907D5
:104720002130310509F080E08083EF85F889E95B6D
:10473000FD4F1082EF85F889E85BFD4F10820E94E3
:10474000560AEF85F889E75BFD4F81E020910C0860
:1047500030910D082130310509F080E080830E94FE
:10476000560AEF85F889E65BFD4F81E0209110083D
:10477000309111082130310509F080E080830E94DA
:10478000560AEF85F889E55BFD4F81E0209114081A
:10479000309115082130310509F080E080830E94B6
:1047A000560AEF85F889E35CFD4F81E020919C0972
:1047B00030919D092130310509F080E080830E940D
:1047C000560AEF85F889E25CFD4F81E02091A0094F
:1047D0003091A1092130310509F080E080830E94E9
:1047E000560AEF85F889E15CFD4F81E02091A4092C
:1047F0003091A5092130310509F080E080830E94C5
:10480000560A0F8518890F591D4F809134089091D1
:104810003508A0913608B0913708F801808391835C
:10482000A283B3830E94560AEF84F888FBE9EF1A4B
:10483000FDEFFF0A8091380890913908A0913A085D
:10484000B0913B08F70180839183A283B3830E94D8
:10485000560A80913C0890913D08A0913E08B09185
:104860003F082F85388927593D4FF901808391836F
:10487000A283B383F8014081518162817381141650
:1048800015061606170644F041E050E060E070E0BF
:104890004083518362837383F70140815181628138
:1048A0007381141615061606170644F041E050E011
:1048B00060E070E0408351836283738318161906A9
:1048C0001A061B064CF081E090E0A0E0B0E0F90190
:1048D00080839183A283B383D9018D909D90AD9005
:1048E000BC90F701C080D180E280F380D8014D9068
:1048F0005D906D907C900E94801BFC0140825182F3
:1049000062827382C482D582E682F7828086918633
:10491000A286B386EF85F889E35CFD4FB081B98349
:10492000EF85F889EF5CFD4F80819181A281B38191
:104930004F855889475B5D4FFA01F081FB834F85B6
:1049400058894E5A5D4FFA01F081FA834F85588994
:104950004D5B5D4FFA01F081FF834F8558894A5BBB
:104960005D4FFA01F081F8874F855889415B5D4FB3
:10497000FA01F081F9874F855889445B5D4FFA0150
:10498000F081FA87EF85F889E25DFD4F2080EF85A1
:10499000F889E151FE4F3080EF85F889EB5AFD4FE1
:1049A0004081518162817381EF85F889EE5DFD4F11
:1049B0000081118122813381EF85F889EA5EFD4F04
:1049C000C080D180E280F380EF85F889E65FFD4FFB
:1049D00080809180A280B380EF85F889EE50FE4FF1
:1049E0004080518062807380EF85F88940A651A68F
:1049F00062A673A684A695A6A6A6B7A6C0AAD1AAA3
:104A0000E2AAF3AA04AB15AB26AB37AB40AF51AF6C
:104A100062AF73AF34AE25AE2A8525A3398536A3A0
:104A20004A8147A340E450E060E070E0E05CFF4F63
:104A300040835183628373832885EF85F88926AF8D
:104A40003F8137AFAF014C5B5F4F2B81FA01208371
:104A5000EF85F889EB5BFF4F80839183A283B3835B
:104A6000EF85F889E75BFF4F39813083AF85B889DF
:104A700055968D919C9156978633910589F483EED6
:104A800090E3FD01E658FF4F9183808332961182B7
:104A9000108281EE90E3369691838083329630C007
:104AA0008C33910589F48BED90E3EF85F889E65816
:104AB000FF4F91838083EF85F889E458FF4F11827F
:104AC000108289ED90E312C08E97E1F483ED90E3BC
:104AD000EF85F889E658FF4F91838083EF85F88949
:104AE000E458FF4F118210828DEC90E3EF85F88936
:104AF000EE57FF4F91838083EF85F889EC57FF4F86
:104B000011821082EF85F889838D948D4A97D1F4B4
:104B10008FED90E3E258FF4F91838083EF85F88912
:104B2000E058FF4F118210828DED90E3EF85F889F8
:104B3000EA57FF4F91838083EF85F889E857FF4F4D
:104B400011821082EF85F889E25CFD4F2081298374
:104B5000EF85F889EB5CFD4F408051806280738067
:104B6000EF85F889E65BFD4F30813B83EF85F8895F
:104B7000ED5AFD4F9081EF85F889EC5BFD4F408148
:104B80004F83EF85F889E95BFD4F50815887EF85AA
:104B9000F889E05BFD4F8081EF85F889E35BFD4F8D
:104BA000A081AA87EF85F889E15DFD4F2080EF8520
:104BB000F889E051FE4F3080EF85F889E75AFD4FC4
:104BC00020813181428153812B873C874D875E87CD
:104BD000EF85F889EA5DFD4F4081518162817381E3
:104BE000EF85F889E65EFD4FC080D180E280F380DA
:104BF000EF85F889E25FFD4F80809180A280B380CD
:104C0000EF85F889E657FF4F2F8538892A503E4FA8
:104C1000D9010D911D912D913C91008F118F228F03
:104C2000338F848E958EA68EB78EC0A2D1A2E2A2BB
:104C3000F3A244A355A366A377A32B853C854D859A
:104C40005E8520A731A742A753A734A625A63A859B
:104C5000358B868B978B80E490E0A0E0B0E080AB52
:104C600091ABA2ABB3AB488546A75F8157A78B81B9
:104C700084AB45AA56AA67AA70AE998191AF858187
:104C800096818633910589F483EE90E3AF85B889E8
:104C9000AC50BF4F8D939C93AF85B889AA50BF4F3E
:104CA0001D921C9281EE90E326C08C33910589F40D
:104CB0008BED90E3AF85B889AC50BF4F8D939C933B
:104CC000AF85B889AA50BF4F1D921C9289ED90E321
:104CD00012C08E97E1F483ED90E3AF85B889AC50B4
:104CE000BF4F8D939C93AF85B889AA50BF4F1D923B
:104CF0001C928DEC90E3AF85B889A450BF4F8D9383
:104D00009C93AF85B889A250BF4F1D921C9283859A
:104D100094854A97D9F48FED90E3EF85F889E850B0
:104D2000FF4F91838083EF85F889E650FF4F118212
:104D300010828DED90E3EF85F889F3959183808360
:104D4000EF85F889EE5FFE4F11821082EF85F889BA
:104D5000E15CFD4FA081A9832F853889275C3D4FF9
:104D6000D9018D919D910D90BC91A02D8B839C8339
:104D7000AD83BE83EF85F889E55BFD4FB081BA83D3
:104D8000EF85F889EC5AFD4F20812F83EF85F88954
:104D9000EB5BFD4F30813887EF85F889E85BFD4F8D
:104DA00040814987EF85F889EF5AFD4F2080EF85D4
:104DB000F889E25BFD4F3080EF85F889E05DFD4FBB
:104DC0003081EF85F889EF50FE4F2081EF85F8891B
:104DD000E35AFD4F80819181A281B381EF85F889EB
:104DE000E65DFD4F4081518162817381EF85F889D5
:104DF000E25EFD4FC080D180E280F380EF85F889CC
:104E0000EE5EFD4F80809180A280B3800F8518896F
:104E10000C5F1E4FEF85F889E650FE4F40805180B1
:104E200062807380F801408E518E628E738E848E04
:104E3000958EA68EB78EC0A2D1A2E2A2F3A244A301
:104E400055A366A377A380A791A7A2A7B3A724A77A
:104E500035A7358A268A2F81278B80E490E0A0E051
:104E6000B0E080AB91ABA2ABB3AB298526A7388568
:104E700037A74A8144AB8B819C81AD81BE8185ABD4
:104E800096ABA7ABB0AF298121AF858196818633E0
:104E9000910589F483EE90E3EF85F889E259FE4F9E
:104EA00091838083EF85F889E059FE4F118210824B
:104EB00081EE90E326C08C33910589F48BED90E36D
:104EC000EF85F889E259FE4F91838083EF85F88959
:104ED000E059FE4F1182108289ED90E312C08E9747
:104EE000E1F483ED90E3EF85F889E259FE4F918379
:104EF0008083EF85F889E059FE4F118210828DEC96
:104F000090E3EF85F889EA58FE4F91838083EF851F
:104F1000F889E858FE4F11821082D8011B968D91B6
:104F20009C911C974A97E1F48FED90E3EF85F88907
:104F3000EE58FE4F91838083EF85F889EC58FE4F41
:104F4000118210828DED90E3EF85F889E658FE4FCF
:104F500091838083EF85F889E458FE4F1182108297
:104F6000EF85F889E05CFD4F20818F859889409618
:104F7000222319F00E94313202C00E941F32EF85B5
:104F8000F889EF5BFD4F20818F85988986579F4F69
:104F9000222319F00E94313202C00E941F32EF8595
:104FA000F889EE5BFD4F80818823D9F0C8016096B7
:104FB0000FB6F894DEBF0FBECDBFDF91CF911F912A
:104FC0000F91FF90EF90DF90CF90BF90AF909F90A8
:104FD0008F907F906F905F904F903F902F900C94A8
:104FE0003132C80160960FB6F894DEBF0FBECDBF58
:104FF000DF91CF911F910F91FF90EF90DF90CF90B5
:10500000BF90AF909F908F907F906F905F904F90E8
:105010003F902F900C941F32CF92DF92EF92FF922D
:105020000F931F93CF93DF936C017A018B01C0E044
:10503000D0E0CE15DF0589F0D8016D918D01D60144
:10504000ED91FC910190F081E02DC6011995892B1D
:1050500011F47E0102C02196ECCFC701DF91CF9100
:105060001F910F91FF90EF90DF90CF9008950895DA
:1050700080E090E00895FC01538D448D252F30E0B1
:10508000842F90E0821B930B541710F0CF96089555
:1050900001970895FC01918D828D981761F0828DA2
:1050A000DF01A80FB11D5D968C91928D9F5F9F735C
:1050B000928F90E008958FEF9FEF0895FC01918DFE
:1050C000828D981731F0828DE80FF11D858D90E06B
:1050D00008958FEF9FEF0895FC01918D228D892F08
:1050E00090E0805C9F4F821B91098F7399270895F0
:1050F0008BEA9BE0F1DF21E0892B09F420E0822F8D
:105100000895FC01848DDF01A80FB11DA35ABF4F84
:105110002C91848D90E001968F739927848FA689B6
:10512000B7892C93A089B1898C9180648C93938DDD
:10513000848D981306C00288F389E02D80818F7DCD
:1051400080830895EF92FF920F931F93CF93DF9385
:10515000EC0181E0888F9B8D8C8D981305C0E889C8
:10516000F989808185FD23C0F62E0B8D10E00F5F3D
:105170001F4F0F731127E02E8C8DE8120BC00FB656
:1051800007FCFACFE889F989808185FFF5CFCE0148
:10519000B8DFF2CF8B8DFE01E80FF11DE35AFF4F10
:1051A000F0820B8FEA89FB898081806207C0EE89DB
:1051B000FF896083E889F98980818064808381E048
:1051C00090E0DF91CF911F910F91FF90EF900895A4
:1051D000CF93DF93EC01888D8823C1F0EA89FB89A6
:1051E000808185FD05C0A889B9898C9186FD0EC096
:1051F0000FB607FCF5CF808185FFF2CFA889B9896A
:105200008C9185FFEDCFCE017CDFE8CFDF91CF9190
:10521000089580E090E0892B19F06ADF811125C0A4
:1052200080E090E0892B41F080E090E0892B21F034
:105230000E94000081111CC080E090E0892B41F0A9
:1052400080E090E0892B21F00E940000811113C0C2
:1052500080E090E0892BA1F080E090E0892B81F044
:105260000E94000081110AC008950E940000D8CF5A
:105270000E940000E1CF0E940000EACF0C940000E1
:10528000089590E0FC013197E231F10508F04EC03D
:105290008827EC59FE4F8F4F0C94C05180918000AD
:1052A0008F7703C0809180008F7D80938000089568
:1052B00080918000877FF9CF84B58F7702C084B555
:1052C0008F7D84BD08958091B0008F7703C0809159
:1052D000B0008F7D8093B0000895809190008F770B
:1052E00007C0809190008F7D03C080919000877FE0
:1052F0008093900008958091A0008F7707C08091DF
:10530000A0008F7D03C08091A000877F8093A000C4
:105310000895809120018F7707C0809120018F7DB3
:1053200003C080912001877F8093200108953FB7BB
:10533000F8948091A70B9091A80BA091A90BB09124
:10534000AA0B26B5A89B05C02F3F19F00196A11DF9
:10535000B11D3FBFBA2FA92F982F8827820F911D0B
:10536000A11DB11DBC01CD0142E0660F771F881F52
:10537000991F4A95D1F708950E94B0520C94FE49A6
:105380000C94FE490F931F93CF93DF93EC01888118
:105390009981009729F02A813B812617370788F4E5
:1053A0008B016F5F7F4F0E94C851009761F0998316
:1053B00088831B830A832C813D81232B11F4FC01FC
:1053C000108281E001C080E0DF91CF911F910F91A9
:1053D00008958F929F92AF92BF92CF92DF92EF92F9
:1053E000FF920F931F930E94FA1962E070E00E94EF
:1053F0009F37892BD1F40E94FA1921E02F931F9235
:105400001F921F921F92812C912CA12CB12CC12C88
:10541000D12C760197018601B701A6010E94330DB8
:105420000F900F900F900F900F9080E090E01F91E1
:105430000F91FF90EF90DF90CF90BF90AF909F9033
:105440008F9008958F929F92AF92BF92CF92DF92EA
:10545000EF92FF920F931F930E94FA191F9221E07F
:105460002F931F921F921F92812C912CA12CB12C53
:10547000C12CD12C760197018601B701A6010E94AB
:10548000330D0F900F900F900F900F9080E090E0F1
:105490001F910F91FF90EF90DF90CF90BF90AF9052
:1054A0009F908F900895EF92FF920F931F93CF9349
:1054B000DF93FC01248135816115710511F480E0D1
:1054C00018C041155105A1F07B01EC018A01020FC2
:1054D000131FB80157DF882391F3288139818C810C
:1054E0009D81B701820F931F0E94C6521D830C83BA
:1054F00081E0DF91CF911F910F91FF90EF90089580
:10550000EF92FF920F931F93CF93DF93CDB7DEB748
:1055100064970FB6F894DEBF0FBECDBF7C01CB0100
:10552000BA018E010F5F1F4F22E044E00E944A49FA
:10553000BC01FC0101900020E9F73197AF01481B45
:10554000590BC701B0DF64960FB6F894DEBF0FBEEB
:10555000CDBFDF91CF911F910F91FF90EF900895F4
:10556000EF92FF920F931F93CF93DF93CDB7DEB7E8
:1055700064970FB6F894DEBF0FBECDBF7C01CB01A0
:10558000BA018E010F5F1F4F22E044E00E944A499A
:10559000BC01FC0101900020E9F73197AF01481BE5
:1055A000590BC70180DF64960FB6F894DEBF0FBEBB
:1055B000CDBFDF91CF911F910F91FF90EF90089594
:1055C000EF92FF920F931F93CF93DF93CDB7DEB788
:1055D0002E970FB6F894DEBF0FBECDBF7C01CB0176
:1055E000BA012AE08E010F5F1F4FA8010E94CD4A29
:1055F000F80101900020E9F73197AF01401B510BF2
:10560000B801C70150DF2E960FB6F894DEBF0FBE6B
:10561000CDBFDF91CF911F910F91FF90EF90089533
:105620006115710549F0FB0101900020E9F7319700
:10563000AF01461B570B37CF80E00895FB01448133
:105640005581608171812FCFEF92FF920F931F934D
:10565000CF93DF93EC017B018A01BA0193DE2881AD
:10566000398181110DC02115310519F0C9010E9440
:10567000FE49198218821D821C821B821A8206C072
:105680001D830C83B701C9010E94C652CE01DF9170
:10569000CF911F910F91FF90EF900895FC018081B1
:1056A00091810C94FE49FC011182108213821282B6
:1056B000158214826115710549F0FB0101900020EB
:1056C000E9F73197AF01461B570BBECF08951F92E4
:1056D0000F920FB60F9211240BB60F922F933F9398
:1056E0004F935F936F937F938F939F93AF93BF93EA
:1056F000EF93FF938BEA9BE004DDFF91EF91BF9165
:10570000AF919F918F917F916F915F914F913F9159
:105710002F910F900BBE0F900FBE0F901F901895FA
:105720001F920F920FB60F9211240BB60F922F9368
:105730008F939F93EF93FF93E091BB0BF091BC0B82
:105740008081E091C10BF091C20B82FD12C090816B
:105750008091C40B8F5F8F732091C50B821751F01E
:10576000E091C40BF0E0E555F44F958F8093C40BA6
:1057700001C08081FF91EF919F918F912F910F90A8
:105780000BBE0F900FBE0F901F901895CF93DF9315
:10579000282F30E0F901E953FB4F8491F901E55CD2
:1057A000FB4FD491F901EF57FB4FC491CC2389F003
:1057B000811167DDEC2FF0E0EE0FFF1FE95DFA4F7E
:1057C000A591B491EC91ED2381E090E021F480E08B
:1057D00002C080E090E0DF91CF9108951F93CF93B6
:1057E000DF93282F30E0F901E953FB4F8491F90151
:1057F000E55CFB4FD491F901EF57FB4FC491CC23EB
:10580000C1F0162F81113DDDEC2FF0E0EE0FFF1FF0
:10581000E35FFA4FA591B4918FB7F894111105C0C9
:105820009C91ED2FE095E92302C0EC91ED2BEC93D8
:105830008FBFDF91CF911F910895CF92DF92EF92AA
:10584000FF920F931F93CF93DF936C018B017A012B
:10585000EC01C256D44F888187FF04C0FB0111823E
:10586000108224C08CE08C9D90018D9D300D112400
:105870008881A901480F511D87FD5A958091E00C40
:1058800090E04817590794F48881A901480F511DE9
:1058900087FD5A95CA01FA01EE0FFF1F8E0F9F1F59
:1058A000FC01E05BF34F808186FD19C088818F5F2A
:1058B00088838CE08C9D90018D9D300D1124888112
:1058C000A901480F511D87FD5A958091E00C90E089
:1058D00048175907B4F488818C303CF112C0888194
:1058E000280F311D87FD3A95F901EE0FFF1F2E0F8E
:1058F0003F1FF901E05BF34F808160E08F736EDF43
:10590000D5CFF80180819181049680349C4918F4A8
:1059100080E49CE904C0F801808191810496F7013C
:10592000918380838FEF888344C0F8014081518147
:105930008881B901680F711D87FD7A95CB01FB0144
:10594000EE0FFF1F8E0F9F1FFC01E05BF34F818165
:105950009281840F951FF701918380838881A9012B
:10596000480F511D87FD5A95CA01FA01EE0FFF1F1E
:105970008E0F9F1FFC01E05BF34F808186FF19C0F3
:105980008881280F311D87FD3A95F901EE0FFF1F21
:105990002E0F3F1FF901E05BF34F808161E08F73B1
:1059A000DF91CF911F910F91FF90EF90DF90CF90FB
:1059B00015CFDF91CF911F910F91FF90EF90DF9066
:1059C000CF900895CF93DF9390E0FC01E55CFB4F0F
:1059D0002491FC01EF57FB4F8491882361F190E003
:1059E000880F991FFC01EF5DFB4FC591D491FC011D
:1059F000E35FFA4FA591B491611109C09FB7F89484
:105A00008881209582238883EC912E230BC06230FD
:105A100061F49FB7F8943881822F8095832388831F
:105A2000EC912E2B2C939FBF06C08FB7F894E88182
:105A30002E2B28838FBFDF91CF910895823091055F
:105A400038F0880F991F880F991F05970197F1F774
:105A500008958F929F92AF92BF92CF92DF92EF9272
:105A6000FF926B017C0163DC4B015C01C114D1042A
:105A7000E104F104E9F05BDCDC01CB018819990950
:105A8000AA09BB09883E9340A105B10578F321E03E
:105A9000C21AD108E108F10888EE880E83E0981E4A
:105AA000A11CB11CC114D104E104F10421F7DECF23
:105AB000FF90EF90DF90CF90BF90AF909F908F902E
:105AC00008952FB7F8946091A30B7091A40B809167
:105AD000A50B9091A60B2FBF08951F920F920FB6A2
:105AE0000F9211242F933F938F939F93AF93BF9364
:105AF0008091A30B9091A40BA091A50BB091A60B44
:105B00003091A20B23E0230F2D3720F40196A11D25
:105B1000B11D05C026E8230F0296A11DB11D2093DB
:105B2000A20B8093A30B9093A40BA093A50BB0930F
:105B3000A60B8091A70B9091A80BA091A90BB091F7
:105B4000AA0B0196A11DB11D8093A70B9093A80BE2
:105B5000A093A90BB093AA0BBF91AF919F918F9186
:105B60003F912F910F900FBE0F901F901895CF92DD
:105B7000DF92EF92FF92CF93DF93EC01603282E0ED
:105B800078070CF03DC077FD06C0653B71052CF031
:105B900064EB70E002C060E070E0898128E830E0EA
:105BA0006901C81AD10887FDD394CC0CDD1CCC0C3C
:105BB000DD1C0D2C000CEE08FF088A8128E532E080
:105BC000281B310987FD3395220F331F220F331F06
:105BD000C901330FAA0BBB0B9C01AD012C193D0968
:105BE0004E095F09DB010E94685024EB30E040E081
:105BF00050E00E944250C20ED31EE41EF51EB601B4
:105C00008881803380F5998148E850E0491B51092B
:105C100097FD5395440F551F440F551F6417750783
:105C200084F09A8128E532E0291B310997FD3395EC
:105C3000220F331F220F331FAB01261737070CF437
:105C4000A90142505109440F551F2FB7F89490E015
:105C5000FC01EE0FFF1F8E0F9F1FFC01E05BF34F57
:105C6000528341832FBFDF91CF91FF90EF90DF9060
:105C7000CF9008951F93CF93DF93EC01162F888167
:105C8000803308F04DC061E0812F9CDE8881E82FD1
:105C9000F0E09F01220F331FE20FF31FE05BF34F91
:105CA0001F739081907C192B108319821A826CE0EB
:105CB0000E94B4519CE0899FB001112440E050E063
:105CC0009A01260F371FF901EE0FFF1F2E0F3F1FFE
:105CD000F901E05BF34F908196FD16C04F5F5F4F77
:105CE0004C30510569F7813001F51092800082E057
:105CF000809381001092850010928400B19A809167
:105D00006F00826080936F00E881F0E0CF01880F20
:105D1000991FE80FF91FE05BF34F80818064808357
:105D20008881DF91CF911F910895823061F41092A4
:105D3000900080939100109295001092940088BB7F
:105D400080937100E1CF833069F41092A00082E06B
:105D50008093A1001092A5001092A40089BB8093AB
:105D60007200D2CF8111D0CF1092200182E08093B7
:105D7000210110922501109224018ABB80937300A7
:105D8000C3CF1F920F920FB60F9211240BB60F9232
:105D90002F933F934F935F936F937F938F939F9333
:105DA000AF93BF93EF93FF9348E251E064E271E059
:105DB00080E090E042DDFF91EF91BF91AF919F9124
:105DC0008F917F916F915F914F913F912F910F90A4
:105DD0000BBE0F900FBE0F901F9018951F920F9241
:105DE0000FB60F9211240BB60F922F933F934F9340
:105DF0005F936F937F938F939F93AF93BF93EF9333
:105E0000FF9348EA50E064EA70E083E090E015DD3B
:105E1000FF91EF91BF91AF919F918F917F916F9182
:105E20005F914F913F912F910F900BBE0F900FBE3E
:105E30000F901F9018951F920F920FB60F9211247A
:105E40000BB60F922F933F934F935F936F937F9374
:105E50008F939F93AF93BF93EF93FF9348E950E0E5
:105E600064E970E082E090E0E8DCFF91EF91BF919F
:105E7000AF919F918F917F916F915F914F913F91E2
:105E80002F910F900BBE0F900FBE0F901F90189583
:105E90001F920F920FB60F9211240BB60F922F93F1
:105EA0003F934F935F936F937F938F939F93AF93A2
:105EB000BF93EF93FF9348E850E064E870E081E01F
:105EC00090E0BBDCFF91EF91BF91AF919F918F91DB
:105ED0007F916F915F914F913F912F910F900BBEEA
:105EE0000F900FBE0F901F90189508950F931F935A
:105EF000CF93DF93FC012081318121153105D1F150
:105F0000EC01822F43DC21E0892B09F420E02B8770
:105F10006A85261729F01E821F82188619860BC0F3
:105F20008E819F81A885B9850196A11DB11D8E83A3
:105F30009F83A887B9870E811F81288539858A812B
:105F40009B81AC81BD81081719072A073B0794F094
:105F500081E06827888142DC0990D881C02D0E94A9
:105F6000D90B40E050E0BE01DF91CF911F910F911E
:105F70000C946D0BDF91CF911F910F910895CF92EB
:105F8000DF92EF92FF920F931F93CF93DF937C01E9
:105F90006B018A01E9010E94560AF601EE0FFF1F0C
:105FA000EE0FFF1FE85AF84F80819181F70191832E
:105FB00080830E94560A000F111F000F111FF80165
:105FC000E85AF84F81E0408151816281738141300C
:105FD00051056105710509F080E0F70182870E9493
:105FE000560ACC0FDD1FCC0FDD1FC85AD84F888151
:105FF0009981AA81BB81F70182839383A483B583AE
:106000001682178210861186DF91CF911F910F9112
:10601000FF90EF90DF90CF90089508952F923F92D8
:106020004F925F926F927F928F929F92AF92BF92A8
:10603000CF92DF92EF92FF920F931F93CF93DF9354
:1060400000D000D0CDB7DEB79E838D834B015A01BF
:106050003A8329831801FC82EB82FA014080518047
:106060006280738020E030E0A901C301B2010E9488
:106070009D51181674F4F6012081318142815381BB
:10608000C301B2010E949F50F50160837183828336
:106090009383ED81FE81E05AFF4F8081F401028DF0
:1060A000138DC088D188E288F388F1014080518047
:1060B00062807380D801A7019601882341F00E9475
:1060C0006850641575058605970544F023C00E9445
:1060D00068504616570668067906E4F4F5014080D4
:1060E00051806280738020E030E04AEF56E4C301C3
:1060F000B2010E94104F87FF0DC020E030E040E861
:106100005FE3C301B2010E94A050F5016083718377
:1061100082839383D801A70196010E946850F10100
:1061200060837183828393830D811E81025C1F4F84
:10613000F80180819181A281B381E981FA81808314
:106140009183A283B383EB81FC8180819181892B30
:1061500041F0C4010E94A40CF80160837183828322
:10616000938326960FB6F894DEBF0FBECDBFDF91A6
:10617000CF911F910F91FF90EF90DF90CF90BF9044
:10618000AF909F908F907F906F905F904F903F90D7
:106190002F9008958FEF9FEF0895EBE0F1E080815D
:1061A000877F80830895EBE0F1E0808188608083C1
:1061B00008958E9808958E9A089514980895149AC3
:1061C000089588980895889A08950C94FE490C942F
:1061D000FE490C94FE490C94FE490C94FE490F9321
:1061E0001F93CF93DF93FB0102A113A1C68DD78D1F
:1061F0000E945A0BC530D105D1F05CF4249749F5C3
:1062000064E070E081EE9CE035DDB80181EE9CE059
:106210001FC0C630D105A1F02B97D9F46BE070E018
:106220008AEE9CE027DDB8018AEE9CE011C065E0B3
:1062300070E084EE9CE01EDDB80184EE9CE008C0B6
:1062400066E070E087EE9CE015DDB80187EE9CE02B
:106250008EDC80E090E0DF91CF911F910F91089547
:106260008F929F92AF92BF92CF92DF92EF92FF9266
:106270000F931F930E94FA191F921F9221E02F93F0
:106280001F921F92812C912CA12CB12CC12CD12CAE
:10629000760197018601B701A6010E94330D0F9088
:1062A0000F900F900F900F9080E090E01F910F9152
:1062B000FF90EF90DF90CF90BF90AF909F908F9026
:1062C00008950E94801B0E94DD1A80E090E00895EE
:1062D00060E0FC01838582CA60E0FC0185817ECAA2
:1062E00061E0FC0183857ACA61E0FC01858176CAA0
:1062F000CF93DF93FB01C68DD78D0E94560ABE0156
:106300000E94130A80E090E0DF91CF9108950895F4
:106310000895089508951F920F920FB60F921124B9
:106320000BB60F922F933F934F935F936F937F938F
:106330008F939F93AF93BF93EF93FF93E0914407A5
:10634000F09145071995FF91EF91BF91AF919F9102
:106350008F917F916F915F914F913F912F910F900E
:106360000BBE0F900FBE0F901F901895CF93DF9329
:10637000EC01FC01E759FF4F1082379781E08083E1
:1063800060E08D812BDA8F859889892B29F060E078
:106390008B85DF91CF9122CADF91CF910895CF9362
:1063A000DF93EC018B89F2D92E8930E082179307B5
:1063B00011F48F8901C080E0DF91CF910895CF93D0
:1063C000DF93EC018989E2D92E8930E082179307A7
:1063D00011F48F8901C080E0DF91CF910895CF93B0
:1063E000DF93EC018DA5882311F061E001C060E02E
:1063F0008F81F4D98EA5882329F08FA5882311F0E9
:1064000061E001C060E08D85DF91CF91E7C9CF9356
:10641000DF93EC018DA5882311F060E001C061E0FD
:106420008F81DCD98EA5882329F08FA5882311F0D0
:1064300060E001C061E08D85DF91CF91CFC9CF933E
:10644000DF93EC0161E08985C9D98EA5882319F015
:1064500061E08F85C3D9C959DF4F1882DF91CF9191
:106460000895CF93DF93EC0160E08985B7D98EA5BD
:10647000882319F060E08F85B1D9C959DF4F81E0D9
:106480008883DF91CF910895CF92DF92EF92FF92B0
:106490000F931F93CF93DF93FC0142AF53AF64AFD1
:1064A00075AFDC01DE964D935D936D937C931397EE
:1064B00014960D931D932D933C931397EC01CA5B97
:1064C000DF4FE88284A9882389F084A5811109C05F
:1064D00037FF0CC01D921D921D921C92139781E0F4
:1064E00006C01016110612061306A4F380E045A993
:1064F00056A967A970AD14161506160617063CF5C1
:1065000091AD992321F10D911D912D913C911397FE
:106510006801790137FF07C0CC24DD247601C01A59
:10652000D10AE20AF30A4C155D056E057F057CF47D
:1065300037FF07C070956095509541955F4F6F4F3D
:106540007F4F4D935D936D937C93139781E0DF01B3
:10655000A15BBF4F1D921D921D921C921397E15A91
:10656000FF4F91E09083DF91CF911F910F91FF90AA
:10657000EF90DF90CF9008950F931F93CF93DF9309
:106580008C01D62FFC018589811109C0C80117DF54
:10659000C82FC80104DFD11108C08C2F06C0C80164
:1065A000FEDEC82FC8010BDFF6CFDF91CF911F9120
:1065B0000F910895CF93DF93EC01FC01E759FF4F52
:1065C00081E0808339978081B297882341F0808170
:1065D0009181A281B3810196A11DB11D07C0808167
:1065E0009181A281B3810197A109B109808391832F
:1065F000A283B383FE01E459FF4F20813181DE0184
:10660000A659BF4FC9019595879520FD03C0ED910F
:10661000FC910DC0FE01E80FF91F0190F081E02D03
:106620002D913C91E20FF31F0190F081E02D8C0F32
:106630009D1F19958F859889892B11F1FE01E059CD
:10664000FF4F20813181DE01A259BF4FC9019595CD
:10665000879520FD03C0ED91FC910DC0FE01E80F70
:10666000F91F0190F081E02D2D913C91E20FF31F75
:106670000190F081E02D8C0F9D1FDF91CF91199437
:10668000DF91CF9108958F929F92AF92BF92CF9258
:10669000DF92EF92FF920F931F93CF93DF93EC0162
:1066A000FC01E15BFF4F60817181828193810E94D7
:1066B000144F6B017C0168A979A98AA99BA90E9442
:1066C000164F9B01AC0160E074E284E799E40E94FC
:1066D00004514B015C01FE01E55AFF4F608171815D
:1066E000828193810E94144F9B01AC01C501B401CA
:1066F0000E9404514B015C018E010D5A1F4F20E096
:1067000030E040E05FE30E94754F9B01AC01C701A0
:10671000B6010E94A0500E947151F80160837183FC
:1067200082839383C95ADF4FA5019401C701B60143
:106730000E94A0500E947151688379838A839B8351
:10674000DF91CF911F910F91FF90EF90DF90CF904D
:10675000BF90AF909F908F9008950F931F93CF930A
:10676000DF93FC01E759FF4F20812223B9F07A978C
:10677000008111812281338138964081518162816B
:106780007381041715072607370710F1EC01EEDDBA
:10679000CE01DF91CF911F910F9175CFFC01E15A8E
:1067A000FF4F20812223A1F0709700811181228167
:1067B00033813496408151816281738104171507BA
:1067C0002607370728F0DF91CF911F910F91F2CE66
:1067D000DF91CF911F910F9108952F923F924F9289
:1067E0005F926F927F928F929F92AF92BF92CF9261
:1067F000DF92EF92FF920F931F93CF93DF93CDB76A
:10680000DEB762970FB6F894DEBF0FBECDBF8C0126
:106810007C0126E4E20EF11CD7018C919801205AEC
:106820003F4FF801EF59FF4F6F01A801425C5F4FE6
:106830004A0114971D01882341F0F80184A5D9016C
:106840008C9381E0F60180832FC0DA014D915D9138
:106850006D917C91F10180819181A281B381BB24F2
:10686000B394481759076A077B070CF0B12CF9015C
:10687000B08277FF07C070956095509541955F4F46
:106880006F4F7F4FB7FF07C0B095A095909581954A
:106890009F4FAF4FBF4F21E0481759076A077B074B
:1068A0000CF420E0D6012C93F401408151816281E7
:1068B0007381411551056105710559F4F801848D05
:1068C000958DA68DB78DE55AFF4F80839183A28366
:1068D000B383F10180819181A281B381F80142AC3F
:1068E00053AC64AC75AC9801215A3F4F590148161E
:1068F00059066A067B0634F4481759076A077B076E
:106900007CF00AC084159505A605B7052CF48417FC
:106910009507A607B70724F0D7018C918823D9F0F3
:10692000F50180818823B9F0D7018C91811105C0D0
:10693000F701808181110FC006C060E0C8011CDE34
:106940008111F6CF17C0D6016C9181E06827C8018C
:1069500013DE882379F0D5011C9260E0C8010CDEBB
:10696000882309F4B3C1F801FE96108211821282C5
:106970001382ACC1D80194962D913D914D915C91BB
:10698000979729833A834B835C8358962D913D9149
:106990004D915C915B972D833E834F8358875C9626
:1069A0002D913D914D915C915F9729873A874B8757
:1069B0005C87F10180819181A281B381F801FE960B
:1069C000C080D180E280F380F80142AD53AD64AD68
:1069D00075ADED59FF4F1082319610823801F5E602
:1069E0006F0E711CF301108298012A593F4FF90173
:1069F0001082329610824C015D01841A950AA60A13
:106A0000B70AB7FE08C0B094A09490948094811CFB
:106A1000911CA11CB11C481759076A077B072CF46D
:106A2000C41AD50AE60AF70A04C0C81AD90AEA0A3B
:106A3000FB0AD501C401B595A795979587958D87D4
:106A40009E87AF87B88BD801A859BF4F1D01F7FCAF
:106A500005C08C149D04AE04BF044CF4F80100A0E2
:106A6000F1A1E02DFA8BE98B81E0D9011BC02D85C6
:106A70003E854F8558892C153D054E055F0508F468
:106A800054C089819A81AB81BC818C159D05AE056E
:106A9000BF0564F42D813E812F5F3F4F3A8B298BD8
:106AA00081E0D3018C93F10180839EC0C701B601C0
:106AB0000E94164F2B013C0169817A818B819C8158
:106AC0000E94164F9B01AC01C301B2010E94045108
:106AD0002B013C016D817E818F81988529853A85C6
:106AE0004B855C85621B730B840B950B0E94164FC4
:106AF0009B01AC01C301B2010E94754F2B013C0107
:106B000069857A858B859C850E94164F9B01AC0117
:106B1000C301B2010E94A0500E946C517A8B698B14
:106B200081E0F801ED59FF4F5CC0D501C401298116
:106B30003A814B815C81821B930BA40BB50BC81669
:106B4000D906EA06FB065CF42D813E812E5F3F4F9D
:106B50003A8B298B81E0F801EB59FF4F42C0C50108
:106B6000B4016C197D098E099F090E94164F2B01F3
:106B70003C0169817A818B819C810E94164F9B0127
:106B8000AC01C301B2010E9404512B013C016D8193
:106B90007E818F81988529853A854B855C85621B2E
:106BA000730B840B950B0E94164F9B01AC01C30124
:106BB000B2010E94754F2B013C0169857A858B8556
:106BC0009C850E94164F9B01AC01C301B2010E943B
:106BD000A0500E946C517A8B698B81E0F801EC59CE
:106BE000FF4F8083D1018C93F80184818823B1F019
:106BF0000E94612DD80112964D905C901397052C40
:106C0000000C66087708DC01CB0184199509A609F8
:106C1000B709893E9340A105B10568F4F801E55A2A
:106C2000FF4F29893A89C901A0E0B0E080839183B0
:106C3000A283B38392CE0E94612DD80113967C93D8
:106C40006E93129786E294E09ED681E296E09BD600
:106C500060E070E0CB01E3D687E296E094D6C7010E
:106C6000B601DDD68DE296E08ED6C501B401D7D649
:106C700083E396E088D64AE06D857E858F85988986
:106C800083D68AE396E07FD669817A818B819C8165
:106C9000C6D680E496E077D669857A858B859C8513
:106CA000BED686E496E06FD66D817E818F81988511
:106CB000B6D68CE496E067D682EA94E064D68989F9
:106CC0009A89D4D68EE993E05ED6A8CF62960FB6A5
:106CD000F894DEBF0FBECDBFDF91CF911F910F9112
:106CE000FF90EF90DF90CF90BF90AF909F908F90EC
:106CF0007F906F905F904F903F902F9008950F93EB
:106D00001F93FC01EA5BFF4F2081211110C03897CF
:106D100000811181228133813496408151816281C9
:106D20007381041715072607370744F404C0FC01D4
:106D300024A5222319F01F910F9169CB1F910F9168
:106D40004ECBFC01138212821482168215821086A9
:106D50001782128611861486138616861586108A67
:106D60001786128A118A148A138ADC01A15ABF4F2E
:106D70001C9212AE13AE14AE15AE91971D921D92D9
:106D80001D921C92139714961D921D921D921C9297
:106D9000139714961C925A961C9211961C92129656
:106DA0001C9211961C9211961C9211961C9211968F
:106DB0001C9211961C9211961C92119684E791E3F5
:106DC00011969C938E93129611961C921E92129677
:106DD00080E791E311969C938E93129611961C92E4
:106DE0001E9212968CE691E311969C938E931296C6
:106DF00011961C921E92129688E691E38D939C93B5
:106E0000E858FF4F11821082089508956E3471057D
:106E10000CF050C06B3471050CF08FC06C327105F2
:106E200054F5693271050CF088C06831710594F42D
:106E30006F3071050CF081C06630710544F462302A
:106E400071050CF07AC0672B09F075C076C06B50E5
:106E500071096EC0623271053CF46F3171050CF03E
:106E60006CC06951710964C0645271096230710566
:106E700008F061C062C06A3371057CF46733710544
:106E80000CF05BC06D3271050CF455C060337105B8
:106E90000CF453C0635371094BC0643471053CF466
:106EA000613471050CF049C06D53710941C06754DC
:106EB00071093EC066387105F4F463387105ECF56C
:106EC0006237710564F46F367105BCF5653671057E
:106ED00094F1683671058CF16956710929C06C37D7
:106EE000710534F46937710544F56357710920C0A1
:106EF0006D5771091DC0603D71057CF46D3C7105D5
:106F0000E4F46439710534F461397105B4F46D58F1
:106F100071090EC0695C71090BC06A3D710534F4DA
:106F2000673D710554F4635D710902C06D5D7109BF
:106F30006330710510F080E0089581E008952F928C
:106F40003F924F925F926F927F928F929F92AF92F9
:106F5000BF92CF92DF92EF92FF920F931F93CF9346
:106F6000DF93CDB7DEB7A3970FB6F894DEBF0FBEA1
:106F7000CDBF9BA38AA37C836B830E94AF208AA191
:106F80009BA10E94C21E8AA19BA10E94901E8AA161
:106F90009BA10E94921E2B813C8121303105C9F1B9
:106FA0002230310509F467C0232B09F097C0AAA04D
:106FB000BBA030E1A30EB11C4AA15BA142585E4FB9
:106FC0005E834D83EAA1FBA1E45BFD4F50815D87A9
:106FD0008AA19BA183599D4F98878F83AAA1BBA1AA
:106FE000A956BD4FBF87AE87EAA1FBA1E755FD4F6C
:106FF000FB8BEA8B2AA13BA127513E4F3C872B8775
:107000004DE850E0598B488B85E190E09A8789875D
:1070100068C0AAA0BBA09AE8A90EB11CAAA1BBA1F6
:10702000A456BE4FBE83AD83EAA1FBA1E35BFD4F37
:10703000B081BD87EAA1FBA1EF58FD4FF887EF8330
:107040002AA13BA127563D4F3F872E874AA15BA12E
:1070500046555D4F5B8B4A8B8AA19BA185519E4F04
:107060009C878B87AEE8B0E0B98BA88BE6E1F0E0B7
:10707000FA87E98736C0AAA0BBA0FCEFAF1AFEEFE3
:10708000BF0A2AA13BA126543E4F3E832D83EAA18D
:10709000FBA1E25BFD4F30813D874AA15BA14B58CC
:1070A0005D4F58874F838AA19BA185569D4F9F872F
:1070B0008E87AAA1BBA1A555BD4FBB8BAA8BEAA108
:1070C000FBA1E351FE4FFC87EB872FE830E0398BC3
:1070D000288B47E150E05A87498703C082E596E054
:1070E0000AC0C5016CD9811104C0C50158D98823D3
:1070F00069F083EE96E047D40E94801B81E090E027
:10710000909347078093460790E0DAC386E294E0C5
:107110003AD481E896E037D4D5018C9175D489E1D1
:1071200097E031D48EE993E02ED481E090E0EB85B6
:10713000FC859183808341E050E0B5018AA19BA149
:107140000E94D81BC5018DD9D5019C968C918501D3
:10715000005A1F4F882331F0C50159D981E0D80169
:107160008C9304C0C5013BD9F80110828D819E81AA
:107170000E94A40CF501FE96608371838283938341
:10718000AF81B8851D921D921D921C921397EAA1A2
:10719000FBA1E359FD4F1082118212821382EAA1F2
:1071A000FBA1EF58FD4F1082118212821382EAA1D7
:1071B000FBA1EB58FD4F108211821282138286E0F0
:1071C00090E0EB85FC859183808346E050E0B5013B
:1071D0008AA19BA10E94D81B41E050E0B5018AA181
:1071E0009BA10E94BD1B412C512C320143948B81E9
:1071F0009C812AA13BA1820F931FAC0147555D4F93
:107200005D8B4C8B2B803C80220C331C220C331C5E
:10721000C10183569D4F280F391F398F288F8B81CD
:107220009C81815A9E4F880F991FAAA1BBA1A80FCC
:10723000B91FBB8FAA8FC10185579D4FEAA1FBA142
:10724000E80FF91FFD8FEC8F910121583D4F3F8FC3
:107250002E8F8AA19BA1820D931DAC014A5E5D4FCA
:1072600059A348A38AA19BA10E946E1EAC89BD8927
:107270008C918823B1F0A10143595D4FEAA1FBA194
:107280004E0F5F1FC88CD98CEA8CFB8C0C8D1D8D2A
:107290002E8D3F8D2E0F3F1F6D817E81C5010E9477
:1072A0000E308BEA9BE00E946C281816190624F019
:1072B0001A82198210E01DC08BEA9BE00E944A28C6
:1072C0008F7D85349105A1F78DE095E05CD30E9418
:1072D000801B21E0DC011C962C9384E693E053D3C1
:1072E0000E94801B0E948A1AE1E0F0E0FA83E983A1
:1072F00011E0C50164D88111D2C2C50150D88111F5
:10730000CEC21111CCC2AE85BF856D917C91072E86
:10731000000C880B990B0E94164F9B01AC01EF816A
:10732000F88560817181828193810E94104F87FF6F
:10733000B6C2C5013FD98AA09BA0820C931CBAEEAD
:107340008B1ABDEF9B0AF401208131814281538168
:1073500060E573EC80E090E00E944250C9010E9419
:107360001E2DD4012D913D914D915C91A3E0B0E093
:107370000E945E509B01AC01C301B2010E944250C9
:10738000672B682B692B39F480E693E0FCD20E94CE
:10739000801B0E948A1AC5010E94B631A8A1B9A11A
:1073A0002D913D914D915C9160E573EC80E090E012
:1073B0000E944250C9010E941E2DBFEF4B1A5B0A6A
:1073C0006B0A7B0AE981FA81EF2B09F44BCF21E0AC
:1073D00030E03A83298342E050E0B5018AA19BA1C5
:1073E0000E94BD1B86E294E0CED281E896E0CBD22B
:1073F000D5018C9109D388E896E0C5D28EE993E057
:10740000C2D2E981FA81EF2BD1F48BE996E0BBD2AD
:1074100082EA94E0B8D288ED94E0B5D289859A8565
:1074200025D382EA94E0AFD28AED94E0ACD2FD8518
:107430008F2F90E01BD30E94801B0E948A1A8AA182
:107440009BA10E94901E8AA19BA10E94921E86E28F
:1074500094E099D281E896E096D2D5018C91D4D26D
:107460008FE996E090D28EE993E08DD2EF81F88596
:107470001082118212821382D5019C968C91850113
:10748000005A1F4F882331F0C5010E94EF31F801E7
:10749000108206C0C5010E94073281E0D8018C939A
:1074A0008D819E810E94A40CF501FE9660837183FC
:1074B00082839383EAA1FBA1E359FD4F10821182DD
:1074C00012821382EAA1FBA1EF58FD4F10821182B4
:1074D00012821382EAA1FBA1EB58FD4F10821182A8
:1074E000128213828D819E810E94A40C6C8B7D8BF5
:1074F0008E8B9F8B412C512C320143948B819C812C
:10750000EAA1FBA18E0F9F1F9C0127553D4F398F8C
:10751000288F2B803C80220C331C220C331CC10191
:1075200083569D4FE80FF91FFB8FEA8F8B819C815B
:10753000815A9E4F880F991F4AA15BA1480F591F7E
:107540005D8F4C8FC10185579D4FAAA1BBA1A80F8C
:10755000B91FBF8FAE8F8AA19BA1820D931DFC0125
:10756000EA5EFD4FF9A3E8A39201215031093A8761
:107570002987490149815A81452B09F0CFC08AA149
:107580009BA10E946E1EA88DB98D8C918823B9F0A5
:10759000910121583D4FEAA1FBA12E0F3F1FA101F0
:1075A00043595D4F4E0F5F1FCA8CDB8CEC8CFD8CFA
:1075B0000E8D1F8D6D817E81C5010E940E308BEA7C
:1075C0009BE00E946C281816190614F010E01DC0EC
:1075D0008BEA9BE00E944A288F7D85349105B1F7A4
:1075E0008DE095E0D0D10E94801B21E0DC011C964B
:1075F0002C9384E693E0C7D10E94801B0E948A1AD4
:10760000E1E0F0E0FA83E98311E029853A852A3048
:10761000310538F4AF81B8851D921D921D921C92E0
:107620001397BD85C501B11146C10E94CF318111AB
:1076300071C0112319F089849A846CC0EE85FF858E
:1076400060817181072E000C880B990B0E94164FE8
:107650009B01AC01AF81B8856D917D918D919C911D
:107660000E94104F87FFE7CFC5010E94DA328AA03F
:107670009BA0820C931CBAEE8B1ABDEF9B0AF401FF
:10768000208131814281538160E573EC80E090E09C
:107690000E944250C9010E941E2DD4012D913D919E
:1076A0004D915C91A3E0B0E00E945E509B01AC0163
:1076B000C301B2010E944250672B682B692B91F4E1
:1076C00080E693E060D10E94801B0E948A1A86E2C5
:1076D00094E059D183EB96E056D1C201C7D18EE92F
:1076E00093E051D1C5010E94B631E8A1F9A12081F2
:1076F00031814281538160E573EC80E090E00E942B
:107700004250C9010E941E2DFFEF4F1A5F0A6F0AF7
:107710007F0A2ACF81EC96E036D104C081E090E068
:107720009A83898386E294E02ED181E896E02BD17A
:10773000D5018C9169D185ED96E025D18EE993E054
:1077400022D18D819E810E94A40CEA89FB89EF2BB6
:10775000A1F0DC01CB012C893D894E895F89821B18
:10776000930BA40BB50BB7FF07C0B095A0959095F0
:1077700081959F4FAF4FBF4F4C0149815A81452B97
:10778000F9F48BE996E0FFD082EA94E0FCD088ED32
:1077900094E0F9D08889998969D182EA94E0F3D09C
:1077A0008AED94E0F0D0B401092C000C880B990B01
:1077B0000E94164F42E05FD10E94801B0E948A1AED
:1077C00085E090E0AB85BC858D939C9345E050E0CF
:1077D000B5018AA19BA10E94D81BC5010E941F323E
:1077E0008AA19BA10E94901E8AA19BA10E94921E29
:1077F000EB81FC81E130F105A1F0E230F10501F10E
:10780000EF2B61F50E94801BC401990CAA0BBB0BE6
:1078100080934C0790934D07A0934E07B0934F076A
:107820001DC00E94801BC401990CAA0BBB0B809346
:10783000500790935107A0935207B09353070EC07F
:107840000E94801BC401990CAA0BBB0B80935407A8
:1078500090935507A0935607B09357070E94801B3B
:107860000E94DD1AAB85BC851D921C9240E050E061
:10787000B5018AA19BA10E94D81B40E050E0B50150
:107880008AA19BA10E94BD1B0E94801BE981FA81F5
:10789000F0934707E093460789819A8111C081ECF4
:1078A00096E071D0C5010E94CF31882309F493CDB1
:1078B000B1E0BD8790CD0E94DF318111BCCEB9CE41
:1078C000A3960FB6F894DEBF0FBECDBFDF91CF9168
:1078D0001F910F91FF90EF90DF90CF90BF90AF90EE
:1078E0009F908F907F906F905F904F903F902F90E0
:1078F0000895CF93DF93FC01E452FE4F4081518104
:107900004115510559F1EC01C052DE4F28813981F2
:1079100088529E4F24173507C8F4FC01808191815D
:10792000009761F0FC01E20FF31F80818A3041F083
:107930008D3029F48EE993E026D002C080E064D037
:107940008881998101969983888308C040E050E03E
:1079500060EA73E00E94242B19821882DF91CF9194
:107960000895009769F0FC0101900020E9F7319734
:10797000AF01481B590BBC018BEA9BE00C940C280F
:1079800080E090E00895EDCF8F929F92AF92BF92EA
:107990000F931F93CF93DF93CDB7DEB7A1970FB6A9
:1079A000F894DEBF0FBECDBF19A2423008F44AE002
:1079B0008E010F5D1F4F842E912CA12CB12CA5019F
:1079C00094010E946E50E62FB901CA0101501109BD
:1079D000EA3014F4E05D01C0E95CD801EC93232B9C
:1079E000242B252B61F7C801BCDFA1960FB6F894B4
:1079F000DEBF0FBECDBFDF91CF911F910F91BF9022
:107A0000AF909F908F900895E091AB0BF091AC0BED
:107A10000190F081E02D682F8BEA9BE01994CF92C2
:107A2000DF92EF92FF92CF93DF9397FF17C06B0126
:107A30007C018DE2E9DFEC0166277727CB016C1929
:107A40007D098E099F094AE09FDF8C0F9D1FDF9102
:107A5000CF91FF90EF90DF90CF9008954AE0DF91B3
:107A6000CF91FF90EF90DF90CF908ECFBC01990F18
:107A7000880B990BD4CF4F925F926F927F928F9227
:107A80009F92AF92BF92CF92DF92EF92FF926B01E3
:107A90007C01B42E9B01AC010E94A151882319F0F6
:107AA00088E397E027C026013701E89477F82FEFA5
:107AB0003FEF4FE75FE7C301B2010E94A15181117F
:107AC0000DC02FEF3FEF4FE75FE7C301B2010E9408
:107AD000104F18161CF48CE397E00CC02FEF3FEF0B
:107AE0004FE75FE4C701B6010E949D5118167CF470
:107AF00080E497E0FF90EF90DF90CF90BF90AF9041
:107B00009F908F907F906F905F904F902ACF2FEF34
:107B10003FEF4FE75FECC701B6010E94104F87FDB2
:107B2000E7CF20E030E0A901C701B6010E94104F65
:107B300087FF08C08DE268DF4C01F7FAF094F7F890
:107B4000F09402C0812C912CA12C60E070E080E0C8
:107B50009FE3AB1441F020E030E040E251E40E94AA
:107B60000451A394F6CF9B01AC01C701B6010E945A
:107B7000A0502B013C010E9471516B017C010E94BD
:107B8000144F9B01AC01C301B2010E949F502B0115
:107B90003C014AE0C701B601F7DE7C01E80CF91CA4
:107BA000BB2021F08EE230DFE80EF91EDB2CDD2059
:107BB00019F120E030E040E251E4C301B2010E943B
:107BC000754F2B013C010E9471514B01A12CB12C2E
:107BD0004AE0C501B401D8DEE80EF91EC501B401C2
:107BE0000E94144F9B01AC01C301B2010E949F503F
:107BF0002B013C01DA94DBCFC701FF90EF90DF90BF
:107C0000CF90BF90AF909F908F907F906F905F903C
:107C10004F900895CF93DF93EC01188A198A1A8A3E
:107C20001B8A60E086E10E94EE2B8C8D8295807F1E
:107C30000E94EC0C61E086E1DF91CF910C94EE2B79
:107C4000789484B5826084BD84B5816084BD85B537
:107C5000826085BD85B5816085BD80916E00816043
:107C600080936E00109281008091810082608093E9
:107C700081008091810081608093810080918000EB
:107C80008160809380008091B10084608093B10016
:107C90008091B00081608093B000809191008260FB
:107CA00080939100809191008160809391008091F8
:107CB00090008160809390008091A1008260809309
:107CC000A1008091A10081608093A1008091A0001B
:107CD00081608093A00080912101826080932101C6
:107CE0008091210181608093210180912001816038
:107CF0008093200180917A00846080937A00809143
:107D00007A00826080937A0080917A00816080930B
:107D10007A0080917A00806880937A001092C10086
:107D200061E08AE10E94E22C61E08BE10E94E22C9A
:107D300061E089E10E94E22C61E08FE00E94E22C88
:107D400061E08EE10E94E22C61E08EE00E94E22C74
:107D500062E085E40E94E22C62E084E40E94E22C6E
:107D600062E080E10E94E22C62E081E10E94E22C6C
:107D700061E080E20E94E22C61E081E20E94E22C5C
:107D800061E08FE10E94E22C62E083E40E94E22C39
:107D900062E082E40E94E22C62E087E10E94E22C31
:107DA00062E088E10E94E22C61E083E20E94E22C22
:107DB00061E084E20E94E22C61E082E20E94E22C17
:107DC00062E081E40E94E22C62E080E40E94E22C06
:107DD00062E08DE10E94E22C62E08CE10E94E22CE4
:107DE00061E088E20E94E22C61E089E20E94E22CDC
:107DF00061E085E20E94E22C61E085E20E94EE2BC8
:107E000061E08DE00E94E22C61E089E00E94E22CBA
:107E100061E088E00E94E22C61E087E00E94E22CB1
:107E200061E08AE00E94E22C61E08CE00E94E22C9A
:107E300062E08FE30E94E22C62E08BE30E94E22C7E
:107E400061E084E00E94E22C61E085E00E94E22C87
:107E500061E086E00E94E22C61E08BE00E94E22C6F
:107E600061E089E10E94EE2B61E08EE00E94EE2B42
:107E700061E08FE10E94EE2B61E082E20E94EE2B36
:107E800084EF91E0909303028093020262E081E329
:107E90000E94E22C61E086E10E94E22C61E086E132
:107EA0000E94EE2B8CB58F7D8CBD8CB5837F8CBDF5
:107EB0008CB58C7F8CBD8DB58E7F8DBDCFB7F89482
:107EC0008091DC0A811127C0E6EBF4E08491E0E7C1
:107ED000F4E09491E82FF0E0EE0FFF1FEF5DFB4F11
:107EE000A591B491EC91E92321F461E085E30E942E
:107EF000EE2B61E085E30E94E22C8CB580618CBDA5
:107F00008CB580648CBD61E084E30E94E22C61E06A
:107F100083E30E94E22C8091DC0A8F5F8093DC0A6D
:107F2000CFBFE091BB0BF091BC0B82E08083E0916E
:107F3000B70BF091B80B1082E091B90BF091BA0B2E
:107F4000D0E1D0831092C30BE091BF0BF091C00B36
:107F500086E08083E091BD0BF091BE0B8081806153
:107F60008083E091BD0BF091BE0B8081886080839F
:107F7000E091BD0BF091BE0B808180688083E09121
:107F8000BD0BF091BE0B80818F7D808364E670E035
:107F900080E090E00E94292D0E94FA190E94891623
:107FA0000E94421E0E940D1E0E94612D6093810B53
:107FB0007093820B8093830B9093840B88EC97E0F3
:107FC0009093450780934407C1E0C0936F00D0931E
:107FD000810010928000C093DF0A80E092E09093CD
:107FE000DE0A8093DD0A909387008093860081E10A
:107FF000809381001092810010928500109284007D
:108000008091DF0A8061809381000E94612D6093DE
:108010007D0B70937E0B80937F0B9093800B0E945F
:10802000612D6093850B7093860B8093870B9093E3
:10803000880B0E94612D6093810B7093820B80935B
:10804000830B9093840B0E94560A80916007909155
:108050006107A0916207B09163070197A105B1057F
:1080600081F40E94560A8091A8079091A907A091D7
:10807000AA07B091AB070197A105B10511F40C94C3
:1080800057480E94560A8091600790916107A0911D
:108090006207B09163070197A105B10581F40E94C1
:1080A000560A8091A4079091A507A091A607B091C8
:1080B000A7070197A105B10511F40C9476480E9419
:1080C000560A8091600790916107A0916207B09174
:1080D00063070197A105B10581F40E94560A8091BA
:1080E000A0079091A107A091A207B091A3070197C3
:1080F000A105B10511F40C94964882E893E043DCA5
:10810000E1E82E2EE2E03E2EF7E7AF2EF2E0BF2EA2
:108110000E94FA190E946E1E0E94612D6093850BC9
:108120007093860B8093870B9093880B0091810B43
:108130001091820B2091830B3091840B6017710793
:108140008207930748F46093810B7093820B8093AE
:10815000830B9093840B2CC0DC01CB01801B910B13
:10816000A20BB30B883E9340A105B10508F108515D
:108170001C4F2F4F3F4F0093810B1093820B209386
:10818000830B3093840B0E94421EEC010E94762FD9
:10819000CE010C960E94762FCE0148960E94762F33
:1081A000CE0184960E94762FCE01C0960E94762F33
:1081B0008BEA9BE00E946C28892B09F4C2C50E94BF
:1081C000612D60937D0B70937E0B80937F0B90935A
:1081D000800B8BEA9BE00E944A2880937C0B982FAF
:1081E0009F7D953479F020917A0B30917B0BF901CA
:1081F000E85BF44F80832F5F3F4F30937B0B2093DE
:108200007A0B06C00E94801B21E0DC011C962C9397
:1082100080917A0B90917B0B8133910564F02AE079
:1082200020937C0BFC01E85BF44F20830196909334
:108230007B0B80937A0B80917C0B20917A0B309191
:108240007B0B8A3039F4C9010197A5E1BBE0E8E472
:10825000FBE004C022333105B4F773C5AF014854C5
:108260005B40481759071CF441914D93F7CFFC012F
:10827000EB5EF44F1082223031050CF45EC583E1D1
:1082800093E081DB82EA94E07EDB81EA93E07BDBB2
:1082900085E19BE078DB81EA93E075DB8EE993E092
:1082A00072DB8AE390E00E946949EC011A821B822A
:1082B0001C821D821E821F82188619861A861B86C2
:1082C0001C861D861E861F86188A198A1A8A1B8A92
:1082D0001C8A1D8A1E8A1F8A188E198E1A8E1B8E62
:1082E0001C8E1D8E1E8E1F8E18A219A21AA21BA2F2
:1082F0001CA21DA21EA21FA218A619A61AA61BA682
:108300001CA61DA61EA61FA618AA19AA1AAA1BAA51
:108310001CAA1DAA1EAA1FAA18AE19AE6AE072E016
:1083200085E19BE00E94994A8C01FC018081865482
:10833000823008F027C163EA73E0C8010E94BD5291
:10834000892B09F4D3C066EA73E0C8010E94BD52CC
:10835000892B09F4CBC06AEA73E0C8010E94BD52C0
:10836000892B09F4C6C06DEA73E0C8010E94BD52B2
:10837000892B09F4BEC061EB73E0C8010E94BD52B5
:10838000892B09F4B9C065EB73E0C8010E94BD52A6
:10839000892B09F4B4C069EB73E0C8010E94BD5297
:1083A000892B09F4ACC06CEB73E0C8010E94BD528C
:1083B000892B09F4A7C060EC73E0C8010E94BD528C
:1083C000892B09F4A2C064EC73E0C8010E94BD527D
:1083D000892B09F49DC068EC73E0C8010E94BD526E
:1083E000892B09F498C06CEC73E0C8010E94BD525F
:1083F000892B09F493C060ED73E0C8010E94BD525F
:10840000892B09F48EC064ED73E0C8010E94BD524F
:10841000892B09F489C068ED73E0C8010E94BD5240
:10842000892B09F484C06CED73E0C8010E94BD5231
:10843000892B09F47FC060EE73E0C8010E94BD5231
:10844000892B09F47AC064EE73E0C8010E94BD5222
:10845000892B09F475C068EE73E0C8010E94BD5213
:10846000892B09F470C06CEE73E0C8010E94BD5204
:10847000892B09F46BC060EF73E0C8010E94BD5204
:10848000892B09F466C064EF73E0C8010E94BD52F5
:10849000892B09F461C068EF73E0C8010E94BD52E6
:1084A000892B09F45CC06CEF73E0C8010E94BD52D7
:1084B000892B09F457C060E074E0C8010E94BD52E6
:1084C000892B09F452C064E074E0C8010E94BD52D7
:1084D000892B09F44DC068E074E0C8010E94BD52C8
:1084E000892B09F448C08FEF9FEF47C080E090E0F0
:1084F00044C081E090E041C08CE190E03EC08DE658
:1085000090E03BC08FE690E038C080E790E035C057
:1085100081E790E032C082E790E02FC083E790E0EF
:108520002CC084E790E029C088E790E026C089E766
:1085300090E023C08AE790E020C083E890E01DC06F
:1085400084E890E01AC08DE890E017C08EE890E0D3
:1085500014C08FE890E011C080E990E00EC081EA7D
:1085600090E00BC085EB90E008C086EB90E005C082
:1085700087EB90E002C088EB90E09093010280933B
:108580000002BBC08FEF9FEF909301028093000227
:10859000B8C0D8018C91883539F4C8010196C6D786
:1085A0006A837B838C839D83F8018081893539F4CC
:1085B000C8010196BBD76E837F8388879987D801CE
:1085C0008C918A3539F4C8010196B0D76A877B87C8
:1085D0008C879D87F8018081813449F4C801019618
:1085E000A5D70E946C516E877F87888B998BD801A5
:1085F0008C91823449F4C801019698D70E946C513D
:108600006A8B7B8B8C8B9D8BF8018081833449F442
:10861000C80101968BD70E946C516E8B7F8B888F1F
:10862000998FD8018C91833539F4C80101967ED792
:108630006A8F7B8F8C8F9D8FF8018081803549F404
:10864000C801019673D70E946C516E8F7F8F88A3EB
:1086500099A3D8018C91863549F4C801019666D753
:108660000E946C516AA37BA38CA39DA3F801808117
:10867000873549F4C801019659D70E946C516EA301
:108680007FA388A799A7D8018C91853449F4C801A4
:1086900001964CD70E946C516AA77BA78CA79DA717
:1086A000F8018081843549F4C80101963FD70E94C2
:1086B0006C516EA77FA788AB99ABD8018C918D3494
:1086C00049F4C801019632D70E946C516AAB7BAB6A
:1086D0008CAB9DABF8018081813549F4C8010196CE
:1086E00025D70E946C516EAB7FAB88AF99AF6CE021
:1086F00074E080E090E01DD78C010115110509F0B0
:1087000048CF0E94801BDC011C961C910E94560AD7
:1087100040906C0750906D0760906E0770906F07E7
:10872000CEA8DFA8E8ACF9AC0E94801BC092480735
:10873000D0924907E0924A07F0924B0780910002DD
:10874000909101028230910508F426C59C012F56B4
:1087500031092530310508F41FC5992493948437D5
:10876000910509F0912C112371F08D36910559F086
:108770009C01285731092330310528F0855B910988
:10878000039708F0D0C20E94560A8091600790912A
:108790006107A0916207B09163070197A105B10538
:1087A00029F0992019F08FEF92E0BFC2209719F4B9
:1087B0008BEF92E0BAC2E0900002F0900102BFEFAE
:1087C000EB16FB06A9F3E114F104B9F48091E00A79
:1087D0009091E10A892B61F482E090E07AD523E15F
:1087E00032E0FC01318320839093E10A8093E00A18
:1087F0000091E00A1091E10A6EC0FCE1EF16F1046D
:10880000B9F48091E20A9091E30A892B61F482E045
:1088100090E05FD52DE132E0DC012D933C93909305
:10882000E30A8093E20A0091E20A1091E30A53C03E
:10883000BDE6EB16F104B9F48091E40A9091E50AE3
:10884000892B61F482E090E044D527E232E0FC011C
:10885000318320839093E50A8093E40A0091E40A2F
:108860001091E50A53C0FFE6EF16F104B9F48091C8
:10887000E60A9091E70A892B61F482E090E029D51D
:1088800021E332E0DC012D933C939093E70A80933F
:10889000E60A0091E60A1091E70A53C000E010E0F2
:1088A000B0E7EB16F104B9F48091E80A9091E90A77
:1088B000892B61F482E090E00CD52BE332E0FC01DF
:1088C000318320839093E90A8093E80A0091E80AB3
:1088D0001091E90A6CC0F1E7EF16F104B9F4809148
:1088E000EA0A9091EB0A892B61F482E090E0F1D4DE
:1088F00025E432E0DC012D933C939093EB0A8093C6
:10890000EA0A0091EA0A1091EB0A6CC0B2E7EB1692
:10891000F104B9F48091EC0A9091ED0A892B61F48D
:1089200082E090E0D6D42FE432E0FC013183208352
:108930009093ED0A8093EC0A0091EC0A1091ED0AF5
:108940006AC0F3E7EF16F104B9F48091EE0A909152
:10895000EF0A892B61F482E090E0BBD429E532E094
:10896000DC012D933C939093EF0A8093EE0A0091E3
:10897000EE0A1091EF0A68C0B4E7EB16F104B9F4FF
:108980008091F00A9091F10A892B61F482E090E0E5
:10899000A0D423E632E0FC01318320839093F10AD6
:1089A0008093F00A0091F00A1091F10A68C0F8E78C
:1089B000EF16F104B9F48091F20A9091F30A892B31
:1089C00061F482E090E085D42DE632E0DC012D9365
:1089D0003C939093F30A8093F20A0091F20A10916B
:1089E000F30A68C0B9E7EB16F104A9F48091F40A20
:1089F0009091F50A892B51F482E090E06AD4FC0151
:108A0000B182A0829093F50A8093F40A0091F40A4F
:108A10001091F50A6AC0FAE7EF16F104A9F4809103
:108A2000F60A9091F70A892B51F482E090E051D434
:108A3000DC012D923C929093F70A8093F60A009104
:108A4000F60A1091F70A6CC0BDE8EB16F104B9F410
:108A50008091F80A9091F90A892B61F482E090E004
:108A600038D42BE832E0FC01318320839093F90A5B
:108A70008093F80A0091F80A1091F90A6CC03EE858
:108A8000E316F104B9F48091FA0A9091FB0A892B5C
:108A900061F482E090E01DD4E5E9F2E0DC01ED93C1
:108AA000FC939093FB0A8093FA0A0091FA0A1091C2
:108AB000FB0A6CC0FFE8EF16F104B9F48091FC0AE0
:108AC0009091FD0A892B61F482E090E002D4EFE9F5
:108AD000F2E0DC01ED93FC939093FD0A8093FC0A95
:108AE0000091FC0A1091FD0A6CC0F0E9EF16F10448
:108AF000B9F48091FE0A9091FF0A892B61F482E01B
:108B000090E0E7D3E9EAF2E0DC01ED93FC93909387
:108B1000FF0A8093FE0A0091FE0A1091FF0A6CC0C2
:108B2000F1EAEF16F104B9F48091000B9091010B7A
:108B3000892B61F482E090E0CCD3E3EBF2E0DC013E
:108B4000ED93FC939093010B8093000B0091000B2D
:108B50001091010B6BC0F5EBEF16F104B9F48091A5
:108B6000020B9091030B892B61F482E090E0B1D36A
:108B7000EDEBF2E0DC01ED93FC939093030B80931B
:108B8000020B0091020B1091030B50C0F6EBEF1695
:108B9000F104B9F48091040B9091050B892B61F4D9
:108BA00082E090E096D3E7ECF2E0DC01ED93FC93F9
:108BB0009093050B8093040B0091040B1091050B0F
:108BC00035C0F7EBEF16F104B9F48091060B9091E4
:108BD000070B892B61F482E090E07BD3E1EDF2E0BA
:108BE000DC01ED93FC939093070B8093060B0091AF
:108BF000060B1091070B1AC0F8EBEF16F104B1F455
:108C00008091080B9091090B892B61F482E090E030
:108C100060D3E5EEF2E0DC01ED93FC939093090B59
:108C20008093080B0091080B1091090B0115110599
:108C300089F48BEF92E00E94C33C0E94801B0E944B
:108C40008A1A80E194E00E94B13C8EE993E00E9490
:108C5000B13C71C087EF92E00E94C33C0E94801B30
:108C60000E948A1A0E94801B1092470710924607A2
:108C7000E12CF12CFFEFEF1AFF0A21E0E216F104DC
:108C800041F083EF92E00E94C33C0E94801B0E944F
:108C90008A1AD801ED91FC910480F581E02DBE0186
:108CA000C80119950E94801BC0904607D0904707C5
:108CB0000E94801BFC018485E114F104D9F281112A
:108CC0000AC0E414F5043CF4C114D10421F0F2E02C
:108CD000CF16D10479F68BEA9BE00E946C28181617
:108CE00019062CF48BEA9BE00E944A28F4CFCD2889
:108CF00009F43CC2992009F43CC20E94560A8091B2
:108D0000680790916907A0916A07B0916B07019776
:108D1000A105B10509F02DC20E94801B21E0DC01F4
:108D20001C962C9326C283E093E00E94C33C0E94D1
:108D3000801B0E948A1ACE0161D310927B0B109285
:108D40007A0B8091140B8111AAC00E94801BFC0138
:108D50008485882309F4A3C00E94FA19EC01FC0160
:108D6000E253FD4F108240960E941F32CE0186577B
:108D70009F4F0E941F32CE018C5F9E4F0E941F3278
:108D80000E94D90B7C018C01075C1F4FC1E0D0E031
:108D90006801F8E3CF1AD108D6018C918823D9F065
:108DA00086E294E00E94C33C8AE294E00E94C33CC5
:108DB000CE010E94363D8EE993E00E94C33C60E004
:108DC0008C2F0E94EE2B40E050E0BE01C7010E94B4
:108DD0006D0BF6011082D8018C918823F9F086E2A0
:108DE00094E00E94C33C81E494E00E94C33CCE0125
:108DF0000E94363D8EE993E00E94C33C61E08C2FD7
:108E00000E94E22C60E08C2F0E94EE2B41E050E0AB
:108E1000BE01C7010E946D0BF801108221960F5F01
:108E20001F4FC533D10509F0B3CF0E945A0B809173
:108E3000E10C90E09C01220F331F820F931FFC0175
:108E4000E05BF34F80818F7B80838091E40C90E026
:108E50009C01220F331F820F931FFC01E05BF34F35
:108E600080818F7B80838091E70C90E09C01220FB2
:108E7000331F820F931FFC01E05BF34F80818F7BD8
:108E800080838091EA0C90E09C01220F331F820FB7
:108E9000931FFC01E05BF34F80818F7B80830E94F6
:108EA000801BDC011C968C918093140BC091120BDB
:108EB000D091130B0E94560AFC0182819381C8173E
:108EC000D90799F00E94560ADC0112968D919C9167
:108ED00013979093130B8093120B0E94FA190E9420
:108EE00089160E94421E0E940D1E0E94612D6093F1
:108EF0000E0B70930F0B8093100B9093110B00913E
:108F00007D0B10917E0B20917F0B3091800B6017B1
:108F100071078207930708F4BDC0AB01BC01401B79
:108F2000510B620B730B8091020290910302092E88
:108F3000000CAA0BBB0B84179507A607B70708F010
:108F4000B3C00E94801BFC018485882319F08FE048
:108F500093E002C08BE093E00E94C33C0E94801B20
:108F60000E948A1A0E94FA19EC01FC01E755FD4F94
:108F70008081882341F0CE0182589E4F0E94A40C2C
:108F80006B017C0107C0FE01E25BFF4FC080D18016
:108F9000E280F3800E94801BC0924C07D0924D0764
:108FA000E0924E07F0924F07FE01E655FD4F80819B
:108FB000882341F0CE0184569E4F0E94A40C6B0181
:108FC0007C0107C0FE01E853FF4FC080D180E280E2
:108FD000F3800E94801BC0925007D0925107E0920C
:108FE0005207F0925307FE01E555FD4F808188231B
:108FF00041F0CE0186549E4F0E94A40C6B017C016F
:1090000006C0CE5BDE4FC880D980EA80FB800E941C
:10901000801BC0925407D0925507E0925607F092F9
:1090200057070E94801B0E94DD1A0E94FA190E94B5
:10903000661C0E94801B0E94C61D0E94801B0E940D
:109040009C1A0E94560A8091600790916107A09136
:109050006207B09163070197A105B10541F087E070
:1090600093E00E94C33C0E94801B0E948A1A809158
:109070000A0B90910B0BA0910C0BB0910D0B01966C
:10908000A11DB11D80930A0B90930B0BA0930C0BA9
:10909000B0930D0B0E94612D60937D0B70937E0B3E
:1090A00080937F0B9093800B0E94092931C887E53C
:1090B00094E00E94C33C0E94FA19CF931F921F9222
:1090C0001F921F92812C912CA12CB12CC12CD12C40
:1090D000760197018601B701A6010E94330D0F901A
:1090E0000F900F900F900F900C9441408FE694E0FA
:1090F0000E94C33C0E94FA191F9221E02F931F92F5
:109100001F921F92812C912CA12CB12CC12CD12CFF
:10911000760197018601B701A6010E94330D0F90D9
:109120000F900F900F900F900C945F4087E894E0A1
:109130000E94C33C0E94FA191F921F9221E02F93B4
:109140001F921F92812C912CA12CB12CC12CD12CBF
:10915000760197018601B701A6010E94330D0F9099
:109160000F900F900F900F900C947D408FEE92E037
:1091700002C08BEE92E00E94C33C0E94801B0E94C2
:109180008A1A0E94801B1092480710924907109279
:109190004A0710924B07CFCD1111C5CD9924939456
:1091A000F2CA88E49CE00C944E2B1092AE0B109205
:1091B000AD0B88EE93E0A0E0B0E08093AF0B90930E
:1091C000B00BA093B10BB093B20B8CE693E09093ED
:1091D000AC0B8093AB0B85EC90E09093B80B809335
:1091E000B70B84EC90E09093BA0B8093B90B80ECB2
:1091F00090E09093BC0B8093BB0B81EC90E090933C
:10920000BE0B8093BD0B82EC90E09093C00B8093DB
:10921000BF0B86EC90E09093C20B8093C10B109231
:10922000C40B1092C50B1092C60B1092C70B82E0B4
:1092300090E04FD02EE733E0FC0131832083909300
:109240004F0C80934E0C60EA73E088E49CE00E942F
:10925000532B8091E00CA1EEBCE09FEF48EB5BE06C
:10926000803378F48C93282F30E0F901EE0FFF1F44
:109270002E0F3F1FF901E05BF34F528341838F5F55
:1092800001C09C931396FCE0AD3EBF0749F7809365
:10929000E00C0895EF920F931F93CF93DF93E801B3
:1092A00047FD02C034E001C034E1E42F440FFF0B5E
:1092B000F7FF03C0F195E195F109E32E022F2E2F60
:1092C000AE01B3D1CE01DF91CF911F910F91EF90FD
:1092D0000895CF93DF938230910510F482E090E0FF
:1092E000E091F10CF091F20C20E030E0C0E0D0E031
:1092F000309711F14081518148175907C0F0481744
:10930000590761F482819381209719F09B838A83A6
:109310002BC09093F20C8093F10C26C021153105DF
:1093200019F04217530718F49A01BE01DF01EF014B
:109330000280F381E02DDCCF2115310509F1281BD6
:10934000390B2430310590F412968D919C9113972E
:109350006115710521F0FB019383828304C0909312
:10936000F20C8093F10CFD01329644C0FD01E20F36
:10937000F31F81939193225031092D933C933AC06E
:109380002091EF0C3091F00C232B41F42091060238
:10939000309107023093F00C2093EF0C20910402DF
:1093A000309105022115310541F42DB73EB74091AA
:1093B000080250910902241B350BE091EF0CF0914B
:1093C000F00CE217F307A0F42E1B3F0B2817390708
:1093D00078F0AC014E5F5F4F2417350748F04E0F11
:1093E0005F1F5093F00C4093EF0C8193919302C058
:1093F000E0E0F0E0CF01DF91CF9108950F931F934C
:10940000CF93DF93009709F48CC0FC01329713824D
:1094100012820091F10C1091F20C0115110581F4EA
:1094200020813181820F931F2091EF0C3091F00C3D
:109430002817390779F5F093F00CE093EF0C71C021
:10944000D80140E050E0AE17BF0750F412962D91BE
:109450003C911397AD012115310509F1D901F3CFE5
:109460009D01DA013383228360817181860F971F0A
:109470008217930769F4EC0128813981260F371F81
:109480002E5F3F4F318320838A819B819383828328
:10949000452B29F4F093F20CE093F10C42C01396A3
:1094A000FC93EE931297ED01499159919E01240F7F
:1094B000351FE217F30771F480819181840F951FA6
:1094C000029611969C938E938281938113969C931E
:1094D0008E931297E0E0F0E0D80112968D919C9166
:1094E0001397009719F0F8018C01F6CF8D919C919C
:1094F00098012E5F3F4F820F931F2091EF0C309108
:10950000F00C2817390769F4309729F41092F20CFF
:109510001092F10C02C0138212821093F00C00938F
:10952000EF0CDF91CF911F910F9108956627772758
:1095300009C24DEE5CE000C0FA01A191B081009734
:1095400019F41097E1F0CD01DC01CD010D90002060
:1095500011F4C00113C0FB012191222319F0201541
:10956000D9F7F3CFFB012191201519F41E92119622
:1095700006C02223C1F70D900020A1F7D001FA0107
:10958000A193B0830895BB274A3031F4992322F484
:10959000BDE2909581959F4F30C0BB272A3051F492
:1095A000992342F4BDE290958095709561957F4F27
:1095B0008F4F9F4F01C0BB27FA01A62F621771057D
:1095C00081059105330B30FB66F0AA27660F771FE4
:1095D000881F991FAA1FA21710F0A21B639538506D
:1095E000A9F7A05DAA3308F0A95DA19336F7B111E0
:1095F000B1931082CA0104C4BB27FB015527AA27D7
:10960000880F991FAA1FA41710F0A41B839550510F
:10961000B9F7A05DAA3308F0A95DA193009779F787
:10962000B111B1931192CB01EBC34F925F926F9244
:109630007F929F92AF92BF92CF92DF92EF92FF9272
:109640000F931F93CF93DF93CDB7DEB729970FB654
:10965000F894DEBF0FBECDBF6A01122FB02E2BE3F0
:10966000201720F0FF24F394F00E02C0BCE3FB2E81
:109670000F2D27E0AE014F5F5F4FCAD2AC01898149
:10968000982F9970913031F0E1FC06C0E0FE06C0E1
:1096900090E205C09DE203C09BE201C090E0EE2D88
:1096A000E07183FF3CC0911102C083E001C084E0FF
:1096B000811718F4212F281B01C020E0E1110BC0F5
:1096C000F601822F30E2882319F031938150FBCFCD
:1096D000C20ED11C20E0992329F0D6019C93F601FB
:1096E00031966F01C6010396E2FE0AC03EE4D60140
:1096F0003C9341E411964C93119712963C9306C00B
:109700003EE6F601308341E641833283FC01322F8D
:1097100040E2332309F442C041933150FACF82FF33
:1097200044C0911102C083E001C084E0811718F4A5
:10973000212F281B01C020E0E1110BC0F601822F70
:1097400030E2882319F031938150FBCFC20ED11C37
:1097500020E0992329F0D6019C93F60131966F0100
:10976000C6010396E2FE0BC039E4D6013C933EE409
:1097700011963C93119736E412963C9307C039E654
:10978000F60130833EE6318336E63283FC01322F28
:1097900040E2332319F041933150FBCFFC01E20F3B
:1097A000F11D10828EEF9FEFB7C0F1E0911101C063
:1097B000F0E06F2F70E01416150624F49A012F5F65
:1097C0003F4F02C021E030E0260F371FBB2029F0B9
:1097D0006B2D70E06F5F7F4F02C060E070E0260F7E
:1097E000371F612F70E0261737071CF4121B212F3B
:1097F00001C020E03E2D387159F4D601322F60E2CD
:10980000332319F06D933150FBCFC20ED11C20E0F1
:10981000FF2331F0D6019C93B6016F5F7F4F6B0140
:10982000E1110BC0F601922F30E3992319F0319327
:109830009150FBCFC20ED11C20E09F2D940F3A8196
:10984000782F7071A72E84FF03C0313309F4915033
:10985000191624F4993018F098E001C091E0E42F33
:10986000852F57FF02C0E0E080E06E2F782FE0E008
:10987000F0E0AEE29A2E3A01691A71082A01461AFE
:10988000570A0B2D10E01195019511096F3F8FEFCD
:10989000780729F4D6019C92C60101966C014617FF
:1098A000570784F0661677066CF47F01E40CF51C0C
:1098B000A1E0B0E0AC0FBD1FEA0EFB1ED701119670
:1098C000BC9002C090E3B92E615071093196C60177
:1098D00001967C016017710724F0D601BC926C01DF
:1098E000D5CF6417750741F4363320F4353321F4AE
:1098F000A11002C081E3B82EF601B082F701822FD9
:1099000090E2882319F091938150FBCFF701E20F89
:10991000F11D108280E090E029960FB6F894DEBF2A
:109920000FBECDBFDF91CF911F910F91FF90EF90B0
:10993000DF90CF90BF90AF909F907F906F905F909F
:109940004F9008956F927F928F929F92AF92BF92A5
:10995000CF92DF92EF92FF920F931F93CF93DF93FB
:10996000EC017B016115710519F0DB018D939C936E
:109970008E010F5F1F4F7880872D90E021D2892BB9
:1099800011F0E801F5CFBDE27B1205C00F5F1F4F5C
:109990007980C1E008C0EBE27E1204C08E010E5F48
:1099A0001F4F7980C0E06801F1E0CF1AD10843E091
:1099B00050E064EF72E0C6010BD2892BE9F4680134
:1099C00022E0C20ED11C45E050E06FEE72E0C6010D
:1099D000FFD1892B21F4680187E0C80ED11CE11466
:1099E000F10419F0D701CD92DC92C111F9C060E009
:1099F00070E080E89FE7FDC043E050E06CEE72E06D
:109A0000C601E6D1892B51F4E114F10409F4EDC04B
:109A10000E5F1F4FF70111830083E7C0680160E00C
:109A200070E0CB0100E010E0F601D0EDD70DDA30A8
:109A300050F52C2F2260622E2C2F2870C2FF05C0FB
:109A4000211127C00F5F1F4F24C0222311F00150A6
:109A50001109A5E0B0E09B01AC0130D34B015C01E2
:109A6000880C991CAA1CBB1CC501B4016D0F711D8B
:109A7000811D911D6839A9E97A078A07A9E19A072A
:109A800040F0C66005C0DE3F51F4C3FD44C0C8606D
:109A90006C2EBFEFCB1ADB0A7080C62DC5CF2D2FE1
:109AA0002F7D2531C1F540814D3211F4C06106C0D2
:109AB0004B3221F0319621E030E006C03296D601DB
:109AC00011964C9122E030E0A0EDA40FAA3018F0DE
:109AD000E21BF30B20C040E050E04038BCE05B07E5
:109AE0005CF49A01220F331F220F331F420F531FC2
:109AF000440F551F4A0F511D3196DF0111972C91CC
:109B0000A0EDA20FAA3048F3C4FF03C051954195C0
:109B10005109040F151FC1FF07C0E114F10421F022
:109B20003197D701ED93FC937FD1C370C33019F007
:109B30006B017C0106C06B017C01F7FAF094F7F829
:109B4000F09420E030E0A901C701B60169D1882373
:109B500009F443C017FF06C0119501951109CBE028
:109B6000D3E002C0C3E2D3E05E01B8E1AB1AB108B2
:109B70004601BE2DAF2D90E2E92EF12C0E151F05EA
:109B80007CF0FE012591359145915491B4018B2FC4
:109B90009A2FABD14B01B82FA92F0E191F09EECF69
:109BA0002497F594E794CA15DB0541F76401EB2E81
:109BB000FA2E8E2D880F8F2D881F8F3F41F020E0C9
:109BC00030E0A901C701B6012BD1811106C082E2A4
:109BD00090E09093F40C8093F30CC701B60109C098
:109BE00060E070E080E89FEF04C060E070E080EC2F
:109BF0009FE7DF91CF911F910F91FF90EF90DF9042
:109C0000CF90BF90AF909F908F907F906F9008956E
:109C1000283008F027E03327DA01990F311D87FD3E
:109C2000916000966105710539F432602E5F3D93B5
:109C300030E32A95E1F708959F3F30F080387105B1
:109C4000610509F03C5F3C5F3D93913008F080680E
:109C5000911DDF93CF931F930F93FF92EF92192FD4
:109C6000987F9695E92F96959695E90FFF27EF57E0
:109C7000FC4F99273327EE24FF24A701E701059025
:109C80000894079428F4360FE71EF81E491F511D4B
:109C9000660F771F881F991F0694A1F705900794F8
:109CA00028F4E70EF81E491F561FC11D770F881FA5
:109CB000991F661F0694A1F70590079428F4F80EE3
:109CC000491F561FC71FD11D880F991F661F771F79
:109CD0000694A1F70590079420F4490F561FC71F5B
:109CE000D81F990F661F771F881F0694A9F78491C4
:109CF0001095177041F0D695C79557954795F794ED
:109D0000E7941A95C1F7E7E2F3E06894159015918E
:109D100035916591959105907FE27395E118F10A6F
:109D2000430B560BC90BD009C0F7E10CF11E431FC2
:109D3000561FC91FD01D7EF4703311F48A95E6CFEB
:109D4000E894015030F0080F0AF40027021708F4D5
:109D5000202F2395022F7A3328F079E37D932A95DB
:109D6000E9F710C07D932A9589F606949795679533
:109D7000379517951794E118F10A430B560BC90B49
:109D8000D00998F023957E9173957A3308F070E3AB
:109D90007C932013B8F77E9170617D9330F08395AA
:109DA00071E37D9370E32A95E1F71124EF90FF9022
:109DB0000F911F91CF91DF91992787FD909508957D
:109DC0009111F6C0803219F089508550D0F708956E
:109DD000FB01DC014150504088F08D9181341CF032
:109DE0008B350CF4805E659161341CF06B350CF49E
:109DF000605E861B611171F3990B0895881BFCCF7F
:109E0000DC01FC01672F71917723E1F7329704C0E1
:109E10007C916D9370836291AE17BF07C8F308956C
:109E200040D008F481E00895E89409C097FB3EF41F
:109E300090958095709561957F4F8F4F9F4F992397
:109E4000A9F0F92F96E9BB279395F6958795779515
:109E50006795B795F111F8CFFAF4BB0F11F460FFD5
:109E60001BC06F5F7F4F8F4F9F4F16C0882311F02D
:109E700096E911C0772321F09EE8872F762F05C041
:109E8000662371F096E8862F70E060E02AF09A95DC
:109E9000660F771F881FDAF7880F9695879597F9D1
:109EA0000895990F0008550FAA0BE0E8FEEF16166B
:109EB0001706E807F907C0F012161306E407F507BE
:109EC00098F0621B730B840B950B39F40A2661F032
:109ED000232B242B252B21F408950A2609F4A140D5
:109EE000A6958FEF811D811D08950BD07BC06CD08E
:109EF00028F071D018F0952309F05DC062C01124DC
:109F0000A5C081D0A0F3959FD1F3950F50E0551FC8
:109F1000629FF001729FBB27F00DB11D639FAA27BE
:109F2000F00DB11DAA1F649F6627B00DA11D661F0D
:109F3000829F2227B00DA11D621F739FB00DA11D2E
:109F4000621F839FA00D611D221F749F3327A00DE8
:109F5000611D231F849F600D211D822F762F6A2F84
:109F600011249F5750408AF0E1F088234AF0EE0F09
:109F7000FF1FBB1F661F771F881F91505040A9F716
:109F80009E3F510570F017C061C05F3FECF3983EF3
:109F9000DCF3869577956795B795F795E7959F5F7D
:109FA000C1F7FE2B880F911D9695879597F9089517
:109FB00099278827089597F99F6780E870E060E007
:109FC00008959FEF80EC089500240A941616170652
:109FD00018060906089500240A941216130614069A
:109FE00005060895092E0394000C11F4882352F0FD
:109FF000BB0F40F4BF2B11F460FF04C06F5F7F4FB5
:10A000008F4F9F4F089557FD9058440F551F59F09B
:10A010005F3F71F04795880F97FB991F61F09F3F55
:10A0200079F087950895121613061406551FF2CF7E
:10A030004695F1DF08C0161617061806991FF1CFCE
:10A0400086957105610508940895E894BB276627F5
:10A050007727CB0197F90895F999FECF92BD81BD7D
:10A06000F89A992780B50895262FF999FECF1FBA3F
:10A0700092BD81BD20BD0FB6F894FA9AF99A0FBE31
:10A0800001960895052E97FB16F400940FD057FD06
:10A0900005D024D007FC02D046F408C05095409566
:10A0A000309521953F4F4F4F5F4F08959095809584
:10A0B000709561957F4F8F4F9F4F089531D0A59F29
:10A0C000900DB49F900DA49F800D911D11240895B3
:10A0D000B7FFF4CFF3DF821B930B0895A1E21A2E92
:10A0E000AA1BBB1BFD010DC0AA1FBB1FEE1FFF1F3C
:10A0F000A217B307E407F50720F0A21BB30BE40B8C
:10A10000F50B661F771F881F991F1A9469F76095D2
:10A110007095809590959B01AC01BD01CF0108958C
:10A12000A29FB001B39FC001A39F700D811D112498
:10A13000911DB29F700D811D1124911D08955058DD
:10A14000BB27AA270ED04ECF3FDF30F044DF20F0F0
:10A1500031F49F3F11F41EF434CF0EF4E095E7FB89
:10A160002ACFE92F50DF80F3BA17620773078407FD
:10A17000950718F071F49EF568CF0EF4E0950B2E5C
:10A18000BA2FA02D0B01B90190010C01CA01A00149
:10A190001124FF27591B99F0593F50F4503E68F1A4
:10A1A0001A16F040A22F232F342F4427585FF3CFE5
:10A1B000469537952795A795F0405395C9F77EF4B6
:10A1C0001F16BA0B620B730B840BBAF09150A1F0FF
:10A1D000FF0FBB1F661F771F881FC2F70EC0BA0F85
:10A1E000621F731F841F48F4879577956795B7950D
:10A1F000F7959E3F08F0B3CF9395880F08F0992705
:10A20000EE0F9795879508950CD0ECCEE4DE40F0E4
:10A21000DBDE30F021F45F3F19F0CDCE511116CFC7
:10A22000D0CEF1DE98F39923C9F35523B1F3951BF2
:10A23000550BBB27AA2762177307840738F09F5F67
:10A240005F4F220F331F441FAA1FA9F333D00E2ED6
:10A250003AF0E0E830D091505040E695001CCAF743
:10A2600029D0FE2F27D0660F771F881FBB1F261708
:10A2700037074807AB07B0E809F0BB0B802DBF01DB
:10A28000FF2793585F4F2AF09E3F510568F093CE09
:10A29000DDCE5F3FECF3983EDCF3869577956795CE
:10A2A000B795F7959F5FC9F7880F911D969587958C
:10A2B00097F90895E1E0660F771F881FBB1F6217AB
:10A2C00073078407BA0720F0621B730B840BBA0B69
:10A2D000EE1F88F7E095089504D06894B111B6CECA
:10A2E000089599DE88F09F5790F0B92F9927B751BC
:10A2F000A0F0D1F0660F771F881F991F1AF0BA954A
:10A30000C9F712C0B13081F0A0DEB1E008959DCE52
:10A31000672F782F8827B85F39F0B93FCCF386953F
:10A3200077956795B395D9F73EF49095809570959C
:10A3300061957F4F8F4F9F4F0895B3DD08F48FEFE6
:10A340000895AFDD880B990B0895DB018F939F93E0
:10A35000B5DEBF91AF91A29F800D911DA39F900D7F
:10A36000B29F900D11240895991B79E004C0991FA4
:10A37000961708F0961B881F7A95C9F7809508955F
:10A38000EE0FFF1F881F8BBF0790F691E02D1994E9
:10A390006F927F928F929F92AF92BF92CF92DF92F5
:10A3A000EF92FF920F931F93CF93DF93EC010097EF
:10A3B00089F4CB01DF91CF911F910F91FF90EF9026
:10A3C000DF90CF90BF90AF909F908F907F906F90D5
:10A3D0000C946949FC01E60FF71F9C0122503109DA
:10A3E000E217F30708F4ABC0D9010D911C91119746
:10A3F00006171707B0F00530110508F49EC0C80114
:10A4000004978617970708F498C002501109061B95
:10A41000170B019311936D937C93CF010E94FE491A
:10A420008CC05B01A01AB10A4C01800E911EA09154
:10A43000F10CB091F20C40E050E0E12CF12C1097BF
:10A4400009F44AC0A815B905D1F56D907C90119713
:10A45000630182E0C80ED11CCA14DB0480F1A301A1
:10A460004A195B096A0182E0C80ED11C1296BC90A1
:10A4700012971396AC91B5E0CB16D10440F0B2829E
:10A48000A38351834083D9016D937C930AC00E5FEF
:10A490001F4FC301800F911FF90191838083EB2D22
:10A4A000FA2FE114F10431F0D7011396FC93EE93E7
:10A4B000129743C0F093F20CE093F10C3EC08D91E3
:10A4C0009C9111974817590708F4AC017D01129629
:10A4D0000D90BC91A02DB3CF8091EF0C9091F00C1A
:10A4E00088159905E1F446175707C8F480910402CE
:10A4F00090910502009741F48DB79EB740910802F4
:10A5000050910902841B950BE817F907C0F4F093EA
:10A51000F00CE093EF0CF901718360830EC0CB0166
:10A520000E9469497C01009751F0A801BE011CD02E
:10A53000CE010E94FE49C70104C0CE0102C080E0E6
:10A5400090E0DF91CF911F910F91FF90EF90DF90FE
:10A55000CF90BF90AF909F908F907F906F90089515
:10A5600081E090E0F89419C0FB01DC0102C0019089
:10A570000D9241505040D8F70895FB01DC018D91B8
:10A58000019080190110D9F3990B0895FB01DC01AA
:10A5900001900D920020E1F7089512E0C2EAD2E0A6
:10A5A00000E005C0802FFE01EBDE2196011DC33ABD
:0CA5B000D10780E00807B1F7F894FFCF56
:10A5BC00FFFF88130000F50C8000200A0D0000003E
:10A5CC00000000681A8516131A00000000691A872B
:10A5DC00161B1D00000000310D2408B207000000FE
:10A5EC00008931E9303031000000000D30C02922E3
:10A5FC002A00000000590B10088B0800000000A175
:10A60C000C1608A30900000000300D2208DB09001D
:10A61C00000000752FBE29E929000000002D0D1C3B
:10A62C0008330B000000000537ED307831000000D6
:10A63C0000A20C1808D40A00000000320D26088471
:10A64C000C00000000A30C1A085A0C000000002F8C
:10A65C000D20086E0C00000000A00C14081F0C004C
:10A66C000000008731E530EF3000000000570B0C84
:10A67C0008F80B000000008A31EB3061310000005B
:10A68C00002E0D1E08B907000000008831E730CA03
:10A69C003000000000580B0E0828085230330052CE
:10A6AC0030320052303700523031005230390052C3
:10A6BC003838005238370052383800523030005297
:10A6CC0038370052303800362E342E322E470000E8
:10A6DC005238350052383400523133005231320086
:10A6EC005231310052373300523732005237310079
:10A6FC005231370052313600523135000100000022
:10A70C0001000000010000005230350052303600CC
:10A71C00523034005238370000000000A2280C28B8
:10A72C003B28E8286C284A285E28000000009F0C73
:10A73C0012085239392041524455494E4F20535436
:10A74C00415254555020434F4D504C4554450D0AE1
:10A75C00002A004730004730300047310047303185
:10A76C000047323800463039004639004631310056
:10A77C004631320046313300463134004631350023
:10A78C004631360046323000463231004632320015
:10A79C004633310046333200463431004634320001
:10A7AC0046343300463434004636310046383100E6
:10A7BC00463832004638330046383400200A0D0043
:10A7CC005239392068616E646C6572203D3D204EB3
:10A7DC00554C4C0D0A005239390020726573657462
:10A7EC0074696E67206469676974616C2070696E46
:10A7FC000020726573657474696E6720616E616C9C
:10A80C006F672070696E0052393920484F4D4520D2
:10A81C005A204F4E20535441525455500D0A005259
:10A82C00393920484F4D452059204F4E2053544123
:10A83C00525455500D0A0052393920484F4D45207D
:10A84C0058204F4E20535441525455500D0A00522B
:10A85C00383320005239392057696C6C207A657274
:10A86C006F2058005239392057696C6C207A657208
:10A87C006F2059005239392057696C6C207A6572F7
:10A88C006F205A0052323100500056005239392094
:10A89C004572726F723A20696E76616C69642070D1
:10A8AC006172616D657465722069640D0A005232C3
:10A8BC00300052343100686F6D650D0A0052393921
:10A8CC0020656D657267656E63792073746F700DAA
:10A8DC000A00523939206572726F720D0A005238B3
:10A8EC0032005239392073746F707065640D0A0030
:10A8FC00523939206572726F722000206465616371
:10A90C00746976617465206D6F746F722058206461
:10A91C00756520746F206D6973736564207374653D
:10A92C007073002064656163746976617465206D71
:10A93C006F746F7220592064756520746F206D6977
:10A94C007373656420737465707300206465616350
:10A95C00746976617465206D6F746F72205A20640F
:10A96C00756520746F206D697373656420737465ED
:10A97C007073005239392074696D656F7574205885
:10A98C0020617869730D0A005239392074696D653C
:10A99C006F7574205920617869730D0A005239392A
:10A9AC002074696D656F7574205A20617869730D18
:10A9BC000A002051005238310020584100205842E2
:10A9CC00002059410020594200205A4100205A428F
:10A9DC000020737461200020637572200020656E66
:10A9EC006420002068616C662000206C656E20007D
:10A9FC00206D696E2000206D6178200020737064DA
:10AA0C0020005239392043616C6962726174696F3C
:10AA1C006E206572726F723A20696E76616C696431
:10AA2C0020617869732073656C65637465640D0AC5
:10AA3C000020617869732000206174207374617246
:10AA4C0074696E6720706F696E7400523233002027
:10AA5C0063616C6962726174696E67206C656E67A4
:10AA6C00746800207374657020636F756E743A207F
:10AA7C0000523939206D6F76656D656E7420646F88
:10AA8C006E650D0A0020617420656E6420706F691C
:10AA9C006E74005239392043616C69627261746959
:10AAAC006F6E206572726F723A20656E64207374DB
:10AABC006F7020616374697665206265666F72657C
:10AACC002073746172740D0A00206D6F76652074AA
:10AADC006F20737461727420666F722063616C698D
:10AAEC0062726174696F6E006E616E00696E6600F1
:04AAFC006F7666000B
:00000001FF
